:100000000C94EA040C9412050C9412050C9412053D
:100010000C9412050C9412050C9412050C94120504
:100020000C9412050C9412050C9412050C941205F4
:100030000C9412050C9412050C9412050C941205E4
:100040000C94091B0C9412050C9464180C943E1823
:100050000C9412050C9412050C9412050C941205C4
:100060000C9496180C941205D11C221CD11CA61FAE
:10007000D61FE91DD61F3C2FD61F9A1F192D1D2DE7
:10008000242D282D2C2D312D352D432D46494E4420
:10009000204D4F44454C004449564552534954590C
:1000A000002020202020202020200053455455509F
:1000B000204D454E55005258353830382076312E77
:1000C000303020204D454E55203200202020202069
:1000D00020202020004641564F52495445530042AB
:1000E000592D4D485A204D4F4445004D414E5541E4
:1000F0004C204D4F44450042414E44205343414E15
:100100004E4552004155544F204D4F4445005258E2
:10011000353830382076312E303020204D454E5540
:10012000203100353934350035383030003533363C
:1001300032004D696E3A20202020204D61783A002F
:100140005253534920534554555000424553543A55
:100150000042414E44205343414E4E4552003539F2
:100160003435003538303000353336320042414EB8
:10017000443A004155544F205345454B204D4F4480
:1001800045004D414E55414C204D4F4445004641A0
:10019000564F52495445204D4F4445002D2D204483
:1001A000454C45544544202D2D004641562043489A
:1001B000414E4E454C3A004348414E4E454C204638
:1001C0005245513A0044454C455445204641564F0E
:1001D00052495445204348414E0042004100414E9F
:1001E00054204200414E542041004155544F004C90
:1001F0004F57205349474E414C0052535349002515
:100200002041004200413A0052454345495645527B
:100210002042005245434549564552204100415530
:10022000544F0044495645525349545900454D5086
:100230005459004641564F524954455300E916D58A
:1002400016C116AD169916851671165D16651678C7
:10025000168B169E16B116C416D716EA1649163511
:100260001621160D16FD161117251739176C168055
:10027000169416A816BC16D016E416F8161A163FD1
:100280001664168916AE16D316F8161D17F2141733
:10029000153C1561158615AB15D015F5154155544E
:1002A0004F205345454B204D4F4445004155544F39
:1002B000204D4F4445204C4F434B004120202020EF
:1002C0002020202000422020202020202020004527
:1002D000202020202020202000462F4169727761B5
:1002E000766500522F52616365626E64004C2F4C3C
:1002F0006F777261636500052A9B29912987291D03
:1003000029132909299F2803290C2916291F29891E
:100310002992299C29052A95288B28812817280F9E
:100320002A192A832A8D2A062910291A2984298E16
:10033000299829022A0C2A1D289028022915298784
:10034000299A290C2A1F2A09261C268E26012713E2
:1003500027862798270B28202020002020200028EF
:10036000292A2B2C2D2E2F131220112110072208A1
:100370001806091905230A1A040B1B03240C1C0276
:100380000D1D25010E1E000F1F26141527161753CD
:10039000415645202620455849540043414C494286
:1003A000524154452052535349005349474E203A35
:1003B00020004F4646004F4E200042454550533ADC
:1003C00020004652455155454E4359004348414E41
:1003D0004E454C2020004F524445523A2000534590
:1003E000545550204D454E550000000000003E5B26
:1003F0004F5B3E3E6B4F6B3E1C3E7C3E1C183C7E72
:100400003C181C577D571C1C5E7F5E1C00183C1856
:1004100000FFE7C3E7FF0018241800FFE7DBE7FF52
:1004200030483A060E2629792926407F05050740DF
:100430007F05253F5A3CE73C5A7F3E1C1C08081CA0
:100440001C3E7F14227F22145F5F005F5F06097FDE
:10045000017F006689956A606060606094A2FFA277
:100460009408047E040810207E201008082A1C0826
:10047000081C2A08081E101010100C1E0C1E0C3030
:10048000383E3830060E3E0E060000000000000028
:100490005F00000007000700147F147F14242A7FE8
:1004A0002A122313086462364956205000080703B5
:1004B00000001C2241000041221C002A1C7F1C2A33
:1004C00008083E0808008070300008080808080086
:1004D0000060600020100804023E5149453E004281
:1004E0007F400072494949462141494D3318141251
:1004F0007F1027454545393C4A4949314121110979
:10050000073649494936464949291E00001400006A
:100510000040340000000814224114141414140084
:100520004122140802015909063E415D594E7C12D0
:1005300011127C7F494949363E414141227F414168
:10054000413E7F494949417F090909013E414151E5
:10055000737F0808087F00417F41002040413F0130
:100560007F081422417F404040407F021C027F7F71
:100570000408107F3E4141413E7F090909063E4182
:1005800051215E7F09192946264949493203017FD5
:1005900001033F4040403F1F2040201F3F40384064
:1005A0003F631408146303047804036159494D43FD
:1005B000007F4141410204081020004141417F0475
:1005C000020102044040404040000307080020545C
:1005D0005478407F284444383844444428384444BC
:1005E000287F385454541800087E090218A4A49C8B
:1005F000787F0804047800447D40002040403D009E
:100600007F1028440000417F40007C047804787CFF
:10061000080404783844444438FC18242418182466
:100620002418FC7C08040408485454542404043F4F
:1006300044243C4040207C1C2040201C3C40304056
:100640003C44281028444C9090907C4464544C4482
:100650000008364100000077000000413608000223
:10066000010204023C2623263C1EA1A161123A404D
:1006700040207A38545455592155557941225454C3
:100680007842215554784020545579400C1E5272BE
:10069000123955555559395454545939555454589B
:1006A0000000457C410002457D420001457C407DC3
:1006B0001211127DF0282528F07C54554500205455
:1006C000547C547C0A097F4932494949323A4444AE
:1006D000443A324A4848303A4141217A3A4240202D
:1006E00078009DA0A07D3D4242423D3D4040403DBE
:1006F0003C24FF2424487E4943662B2FFC2F2BFFEC
:100700000929F620C0887E0903205454794100004D
:10071000447D413048484A32384040227A007A0AC3
:100720000A727D0D19317D2629292F28262929298C
:100730002630484D402038080808080808080838BE
:100740002F10C8ACBA2F102834FA00007B00000824
:10075000142A142222142A14085500550055AA55AB
:10076000AA55AAFF55FF55FF000000FF001010100A
:10077000FF00141414FF001010FF00FF1010F01001
:10078000F0141414FC001414F700FF0000FF00FF25
:100790001414F404FC141417101F10101F101F144D
:1007A00014141F00101010F0000000001F10101093
:1007B000101F10101010F010000000FF101010108B
:1007C0001010101010FF10000000FF140000FF00B8
:1007D000FF00001F10170000FC04F414141710177A
:1007E0001414F404F40000FF00F714141414141487
:1007F00014F700F7141414171410101F101F1414FA
:1008000014F4141010F010F000001F101F0000006E
:100810001F14000000FC140000F010F01010FF1076
:10082000FF141414FF141010101F00000000F0102B
:10083000FFFFFFFFFFF0F0F0F0F0FFFFFF00000010
:100840000000FFFF0F0F0F0F0F3844443844FC4ADD
:100850004A4A347E02020606027E027E026355493F
:1008600041633844443C04407E201E2006027E0240
:100870000299A5E7A5991C2A492A1C4C7201724CC1
:10088000304A4D4D303048784830BC625A463D3E83
:10089000494949007E0101017E2A2A2A2A2A444424
:1008A0005F444440514A444040444A51400000FFA4
:1008B0000103E080FF000008086B6B083612362445
:1008C00036060F090F06000018180000001010006F
:1008D0003040FF0101001F01011E00191D17120009
:1008E0003C3C3C3C000000000000000000240027CD
:1008F000002A0000000000250028002B0000000056
:100900000023002600290004040404040404040253
:10091000020202020203030303030301020408109C
:100920002040800102040810200102040810200069
:10093000000008000201000003040700000000009E
:100940000000002D2D205341564544202D2D0046FA
:100950005245513A20202020204D487A0020204640
:100960004156204348414E3A004348414E3A0053D5
:10097000455454494E475320534156454400534132
:1009800056452053455454494E47530053454C4512
:1009900043544544204641564F524954452043480C
:1009A00000A1A2A3A4A5A6A7A8B1B2B3B4B5B6B737
:1009B000B8E1E2E3E4E5E6E7E8F1F2F3F4F5F6F7AF
:1009C000F8717273747576777811121314151617FF
:1009D0001800783111241FBECFEFD8E0DEBFCDBFA5
:1009E00027E0A2E7B5E001C01D92AD33B207E1F701
:1009F00015E0A0E0B1E0E8ECF9E602C005900D9248
:100A0000A237B107D9F714E0CAEED4E004C02197A9
:100A1000FE010E941E32C93ED107C9F70E94531B36
:100A20000C94E2340C9400000F931F93CF93DF9348
:100A3000DC0155968C915597823071F0833009F125
:100A4000813009F08CC01496ED91FC911597E41B50
:100A5000F50BE21BF30B20C01496ED91FC9115975A
:100A6000CF01861B970BBC01615071091696ED9161
:100A7000FC911797CF01841B950BAC01421B530BC4
:100A80006EC01696ED91FC911797CF01861B970BC0
:100A9000BC0161507109FA0177FD1BC116968D9159
:100AA0009C911797681779070CF013C1F7FF04C0E2
:100AB0002E0F3F1FE0E0F0E014968D919C9115976A
:100AC000AF01420F531F841795071CF49C012E1B86
:100AD0003F0B121613060CF0FCC0CB0177FD0796F6
:100AE00043E0959587954A95E1F79695982F882745
:100AF00097958795E80FF91FE15EFE4F677077279E
:100B000081E090E001C0880F6A95EAF7482F013034
:100B1000110541F088F00230110509F0DAC02E0FFE
:100B20003F1F15C02E0F3F1FE217F30709F4D1C076
:100B30008081842B8193F8CF80952E0F3F1FE21781
:100B4000F30709F4C6C0908198239193F8CFE21778
:100B5000F30709F4BEC0808184278193F8CF77FD25
:100B6000B8C014968D919C911597681779070CF071
:100B7000B0C057FF04C0240F351F40E050E0169668
:100B80008D919C911797FA01E20FF31F8E179F0723
:100B90001CF49C01241B350B121613060CF099C093
:100BA000A22F842F86958695869590E8899F600D63
:100BB000711D1124FB01E15EFE4F4770A9F198E021
:100BC000941B492F50E0EA01C15DDA4F8881291753
:100BD00090F4421B51092FEF30E002C03595279564
:100BE0004A95E2F782230130110541F068F00230A6
:100BF000110589F06EC00130110519F42081822B96
:100C00000CC00130110520F480952081822305C09D
:100C10000230110531F4208182278083A91708F45E
:100C200058C0A91BE058FF4FA83048F10230110509
:100C300059F4EF018A2F988190959883C058DF4F1F
:100C400088508830C0F730C081E00130110509F0CC
:100C500080E08195EF019A2F8883C058DF4F98502C
:100C60009830D0F788EF8A0F86958695869590E81C
:100C7000899FE00DF11D1124E058FF4FA770AA23B2
:100C800041F1B0E0A95DBA4F8C910130110529F016
:100C900038F002301105D1F01CC09081892B18C0AA
:100CA00080959081892314C088EF8A0F8695869558
:100CB000869590E8899FE00DF11D1124E058FF4FC3
:100CC000A77039F0B0E0A95DBA4F8C919081892767
:100CD0008083DF91CF911F910F9108950F931F9300
:100CE000CF93DF93DC01FB0155968C9155978230B1
:100CF00081F0833019F1813051F514968D919C91DA
:100D00001597BC01641B750BAB0141505109BF0124
:100D100081C014966D917C911597CB018E1B9F0B12
:100D2000FC0116968D919C911797BC01641B750B65
:100D3000AB0141505109E21BF30B09C016966D91AE
:100D40007C9117976E1B7F0B621B730B63C057FD63
:100D50001CC116968D919C911797481759070CF056
:100D600014C1F7FF04C02E0F3F1FE0E0F0E014961F
:100D70008D919C911597BF01620F731F861797077E
:100D80001CF49C012E1B3F0B121613060CF0FDC029
:100D9000CA0157FD079663E0959587956A95E1F737
:100DA0009695982F882797958795E80FF91FE15E0C
:100DB000FE4F4770552781E090E001C0880F4A95AB
:100DC000EAF7482F0130110541F088F00230110593
:100DD00009F0DBC02E0F3F1F15C02E0F3F1FE2177B
:100DE000F30709F4D2C08081842B8193F8CF8095DA
:100DF0002E0F3F1FE217F30709F4C7C09081982315
:100E00009193F8CFE217F30709F4BFC080818427DC
:100E10008193F8CF57FDB9C014968D919C91159789
:100E2000481759070CF0B1C077FF04C0260F371FD1
:100E300060E070E016968D919C911797FB01E20F90
:100E4000F31F8E179F071CF49C01261B370B1216ED
:100E500013060CF09AC0A22F862F8695869586954C
:100E600090E8899F400D511D1124FA01E15EFE4F6B
:100E70006770A9F198E0961B492F50E0EA01C15D27
:100E8000DA4F8881291790F4421B51092FEF30E087
:100E900002C0359527954A95E2F782230130110566
:100EA00041F068F00230110589F06FC00130110582
:100EB00019F42081822B0CC00130110520F480959B
:100EC0002081822305C00230110531F42081822760
:100ED0008083A91708F459C0A91BE058FF4FA83018
:100EE00048F10230110559F4EF018A2F988190954D
:100EF0009883C058DF4F88508830C0F731C081E0F8
:100F00000130110509F080E08195EF019A2F888367
:100F1000C058DF4F98509830D0F788EF8A0F8695E9
:100F20008695869560E8869FE00DF11D1124E058B6
:100F3000FF4FA770AA2349F1B0E0A95DBA4F8C9189
:100F40000130110529F038F002301105D9F01DC02B
:100F50009081892B03C0809590818923808315C05F
:100F600088EF8A0F86958695869570E8879FE00DB5
:100F7000F11D1124E058FF4FA77039F0B0E0A95DD2
:100F8000BA4F8C9190818927E9CFDF91CF911F9142
:100F90000F910895FC0177FD9AC0808591856817AF
:100FA00079070CF094C057FD92C08285938548174D
:100FB00059070CF08CC08589823009F07CC084818F
:100FC0009581DC01A61BB70BBD01615071098681BB
:100FD0009781FC01E41BF50BAF01415051090AC098
:100FE000813041F484819581841B950BAB01BC0158
:100FF000615071092130310529F008F122303105A5
:10100000E1F10895FA0157FD3796A3E0F595E795CC
:10101000AA95E1F7F695FE2FEE27F795E7956E0F67
:101020007F1FFB01E15EFE4F4770552781E090E096
:1010300001C0880F4A95EAF79081892B3AC0FA01DE
:1010400057FD379623E0F595E7952A95E1F7F69554
:10105000FE2FEE27F795E7956E0F7F1FFB01E15EF0
:10106000FE4F4770552781E090E001C0880F4A95F8
:10107000EAF78095908189231CC0FA0157FD3796C5
:1010800083E0F595E7958A95E1F7F695FE2FEE2733
:10109000F795E7956E0F7F1FFB01E15EFE4F4770EE
:1010A000552781E090E001C0880F4A95EAF79081CA
:1010B000892780830895833009F092CF86819781B4
:1010C000861B970BBA01AC014150510993CF08958B
:1010D00008952F923F924F925F926F927F928F92DC
:1010E0009F92AF92BF92CF92DF92EF92FF920F93B7
:1010F0001F93CF93DF93CDB7DEB76B970FB6F894FE
:10110000DEBF0FBECDBF4C015A8349831F830E83C0
:10111000FD82EC82CB82DC0158964D915C9159970F
:101120004115510509F0A5C018968D919C9119970C
:10113000681779070CF05AC11A968D919C911B97EC
:10114000E981FA81E817F9070CF050C1D12CCB01E5
:101150003B81F6E03F9F800D911D11241816190662
:101160000CF044C1C60133E0880F991F3A95E1F7AE
:1011700049815A81840F951F181619060CF036C143
:1011800057968C91811103C0203B08F02F5F55E0EA
:10119000259F900111247E876D875B01212CC90159
:1011A000861B970B99878887A981BA811896BB8778
:1011B000AA87B5E02B1641F0E885F985EA0DFB1DFD
:1011C000E751FC4F349001C0312C69807A802301B3
:1011D00030FE12C0D401ED91FC91BB81B13031F4ED
:1011E0000480F581E02D2E813F8118C00684F785AB
:1011F000E02DEE80FF801CC0EC81FD812E813F81BF
:10120000E217F307E1F0D401ED91FC91BB81B1301D
:1012100051F40480F581E02D2C813D81A301B501BD
:10122000C40109950CC00684F785E02DEC80FD8093
:1012300086019601A2016D857E85C40109953694CB
:10124000EFEF6E1A7E0A4C0C5D1C2A853B856216F8
:10125000730609F0BDCF23943FEFA31AB30A4D855F
:101260005E854C0D5D1D5E874D8756E02512A1CF32
:10127000BDC0FA0134963491329785919491231B25
:10128000A7E02A9F800D911D1124FA012591349128
:101290003A8B298BFC0125903490FC0132963491D5
:1012A0003887319644914C873196E491FC0135960C
:1012B000A491319684915B81523050F06A2E0A2EAF
:1012C000000C7708E82F082E000CFF0BFB87EA873D
:1012D000FB81CF2ED12C6C9C90016D9C300D7C9CA1
:1012E000300D1124A901460F571F588B4F871C82C0
:1012F000A12CEA2FAA0FFF0B3B016E0E7F1E588513
:10130000650F711DDB01AE0FBF1FBF8BAE8BE98177
:10131000FA81E80FF11D87FDFA95F98FE88F9C851A
:10132000A91608F063C08A2D90E04A855B85480FB6
:10133000591F4C9D90014D9D300D5C9D300D112429
:10134000A981BA81A20FB31FBE87AD877B8E6A8E3B
:101350004F845888BC81B619BB8BE88DF98DE80F96
:10136000F91FFD8BEC8B8B89FA8D8F0F2A8D3B8DAE
:101370004E895F892417350799F1877041F4C101BF
:101380000196E989FA89E20DF31DB4901C01B7FEBC
:101390001EC0D401ED91FC91BB81B13061F4048099
:1013A000F581E02D2E813F814C895D896A8D7B8D91
:1013B000C40109950CC00684F785E02DEE80FF80FE
:1013C000860196014D855E85B201C4010995BB0C6D
:1013D000EA8DFB8D3196FB8FEA8F4C0C5D1CC3CFE1
:1013E0005C818885580F5C83A39499CF6B960FB668
:1013F000F894DEBF0FBECDBFDF91CF911F910F914B
:10140000FF90EF90DF90CF90BF90AF909F908F9024
:101410007F906F905F904F903F902F900895AF9284
:10142000BF92CF92EF92FF920F931F93CF93DF93D0
:10143000EC01262F888D998D009709F042C06A3003
:1014400069F42C898E859F8538E0239F800D911D3E
:1014500011249F878E871D861C86ACC06D3009F4D1
:10146000A9C08E898823C1F03C898C859D8546E082
:10147000349F800D911D1124488559858417950747
:101480005CF01D861C868E859F85E8E03E9F800D62
:10149000911D11249F878E87EA88FB880889198906
:1014A0004E855F856C857D85CC88CE010E9469085C
:1014B0002C898C859D85F6E02F9F800D911D112430
:1014C00041C06A3079F41D861C862C89FC01369651
:1014D000E4918E859F852E9F800D911D11249F87FD
:1014E0008E8768C06D3009F465C0AC014C5F5F4FFA
:1014F000FA013491631708F45DC03196E491E61760
:1015000008F458C0FA014491362F341BFC0132967E
:10151000A590B490F7E03F9FA00CB11C1124F501F9
:10152000329634913196E491332311F0E1110DC0DC
:10153000F5013496E4912C898C859D85E29F800D80
:10154000911D11249D878C8735C0F50135964491F6
:101550005E89552311F16C89E32FF0E0E40FF11D52
:1015600047FDFA956E9FD0016F9FB00D11244C85F9
:101570005D854A0F5B1FE885F9854E175F076CF0A4
:101580001D861C86FC013696E4918E859F856E9F94
:10159000800D911D11249F878E87EA88FB8808891A
:1015A00019894E855F856C857D85CC88CE010E942A
:1015B0006908BECF81E090E0DF91CF911F910F913C
:1015C000FF90EF90CF90BF90AF900895EF92FF9271
:1015D0000F931F93DC01ED91FC9111971A960D91D9
:1015E0001C911B9718962D913C9119970684F785AD
:1015F000E02D7B0140E050E060E070E009951F9134
:101600000F91FF90EF9008956F927F928F929F922B
:10161000AF92BF92CF92DF92EF92FF920F931F9300
:10162000CF93DF936C015A014801EB013B01620E3D
:10163000731EC615D70574F4D601ED91FC91008494
:10164000F185E02D87019401A501BE01C601099530
:101650002196EFCFDF91CF911F910F91FF90EF90E7
:10166000DF90CF90BF90AF909F908F907F906F90C2
:101670000895EF92FF920F931F93DC01ED91FC917F
:10168000260F371F215031090680F781E02D7801A0
:101690008A0109951F910F91FF90EF900895EF92A5
:1016A000FF920F931F937801DC01ED91FC91240FC1
:1016B000351F8901015011090680F781E02D9B013A
:1016C00009951F910F91FF90EF9008956F927F926F
:1016D0008F929F92AF92BF92CF92DF92EF92FF9242
:1016E0000F931F93CF93DF93EC014B015A016901D4
:1016F0003801E881F9810284F385E02D870109959D
:10170000E881F981A501460D571D41505109028418
:10171000F385E02D9601B401CE010995E881F981A8
:101720000084F185E02D9301A501B401CE01099556
:10173000E881F981C80CD91CB60161507109008497
:10174000F185E02D9301A501CE010995DF91CF919F
:101750001F910F91FF90EF90DF90CF90BF90AF90CF
:101760009F908F907F906F9008952F923F924F920D
:101770005F926F927F928F929F92AF92BF92CF9221
:10178000DF92EF92FF920F931F93CF93DF9300D0DE
:101790001F92CDB7DEB74C017B836A836A01590182
:1017A00017019801241B350B37FF03C03195219594
:1017B0003109C5014A815B81841B950B97FF03C0EA
:1017C00091958195910951E059838217930714F0FF
:1017D00019820BC09A2D8B2D5801092F182F9A8131
:1017E0008B81DB82CA82C92ED82E8A819B81A81662
:1017F000B9065CF49C2D8D2D6801092F182F9A8154
:101800008B81BB82AA82A92EB82E2501AA81BB8119
:101810004A1A5B0A38016C187D0877FE03C0719480
:1018200061947108720157FE03C0BFEFEB1AFB0A07
:10183000F594E794C016D1061CF00FEF1FEF1FC000
:1018400001E010E01CC0D401ED91FC91B98104804D
:10185000F581E02D9101BB23C1F04A815B81B60186
:10186000C4010995E618F708F7FE04C0C00ED11EA2
:10187000E40CF51CEA81FB813196FB83EA834A8103
:101880005B81A416B506FCF604C0A6016A817B81C3
:10189000E7CF0F900F900F90DF91CF911F910F9195
:1018A000FF90EF90DF90CF90BF90AF909F908F9080
:1018B0007F906F905F904F903F902F9008954F9240
:1018C0005F926F927F928F929F92AF92BF92CF92D0
:1018D000DF92EF92FF920F931F93CF93DF93782EB7
:1018E0009AE0F92EC0E0D0E000E010E084E10E9430
:1018F0003F1284E10E943F12080F191F85E10E94E8
:101900003F1285E10E943F12C80FD91FFA94F110CF
:10191000EDCFEAE0F0E0C801BF010E940A329B016E
:10192000CE01BF010E940A328B0180911C018830D8
:1019300061F580911401909115012817390720F461
:10194000309315012093140180911201909113019D
:101950008217930720F43093130120931201809192
:101960000C0190910D010817190720F410930D0137
:1019700000930C0180910A0190910B01801791074F
:1019800020F410930B0100930A01C0901801D0902D
:101990001901E12CF12CC901330FAA0BBB0B9C01DF
:1019A000AD012C193D094E095F09A3E6B0E00E9484
:1019B000A63420911601309117014901A12CB12CB8
:1019C000A50194012C193D094E095F090E94873435
:1019D00069017A018FEFC81AD80AE80AF80AE60105
:1019E0008090100190901101A12CB12CC801110F11
:1019F000AA0BBB0B9C01AD01281939094A095B09E7
:101A0000A3E6B0E00E94A63420910E0130910F01B0
:101A1000890120E030E0A9019801281939094A0913
:101A20005B090E94873449015A018FEF881A980A8E
:101A3000A80AB80A84012FEF721266C0809175055A
:101A4000882321F0823009F452C04EC0B401092C21
:101A5000000C880B990B0E943B332B013C01B60113
:101A6000DD0C880B990B0E943B33A30192010E946D
:101A70002432A30192010E94913220E030E048EC30
:101A800052E40E94CC336B017C0120E030E0A901DC
:101A90000E94C73318161CF4C701B60103C0C70162
:101AA000B60190580E94033364307105BCF08091F8
:101AB00090050C171D0724F4181654F4815006C025
:101AC000C017D1072CF487301CF48F5F80939005EA
:101AD00080919005882341F087304CF47090060186
:101AE00081E078120BC006C07724739403C082E0B3
:101AF000782E04C088B18C7F816003C088B18C7F50
:101B0000826088B97092060121E0721629F08091F6
:101B10001C01883009F0E401C0908C05D0908D053F
:101B2000E0908E05F0908F05C114D104E104F1041A
:101B300029F10E94FD1A20E4C20E2FE1D21EE11C01
:101B4000F11CC616D706E806F906C0F480911C0100
:101B50008930A1F42091060180911E0182131BC0DF
:101B600080918B0590E0AE014C5351098417950785
:101B700094F048585F4F481759076CF01C161D0623
:101B80003CF4CE01C536D105BCF084E690E014C02B
:101B900081E090E011C020931E01C0938B0581E08D
:101BA00090E0A0E0B0E080938C0590938D05A09329
:101BB0008E05B0938F05E2CFDF91CF911F910F91EA
:101BC000FF90EF90DF90CF90BF90AF909F908F905D
:101BD0007F906F905F904F9008958FEF0C945F0C03
:101BE0000E94FD1A60938C0570938D0580938E057D
:101BF00090938F050E94FD1A2091C4063091C5066E
:101C0000621B730B6332710550F483E290E09C0118
:101C1000261B370BB90180E090E00C945612089512
:101C2000CF93DF939C01ADE3B2E040E050E0FD01D3
:101C3000C591D491C217D30711F4842F22C04F5FEE
:101C40005F4F12964033510591F7662349F02F5F9D
:101C50003F4F203747E134075CF028E833E108C004
:101C600021503109283843E1340714F42FE637E1D5
:101C700028173907C1F6283A364110F08FE201C023
:101C800080E0DF91CF910895982F2FE533E080E039
:101C9000F90145915491941731F08F5F2F5F3F4FB9
:101CA0008033B1F780E008959091B606992339F01A
:101CB0008EBD00000DB407FEFDCF8EB5089528E05F
:101CC00030E040E8E091B906F091BA065081909179
:101CD000C006909595239083E091B706F091B806E1
:101CE0009091BF06542F582319F05081952B03C0B3
:101CF0005081909595239083E091B906F091BA06B2
:101D000050819091C006952B9083469521503109C2
:101D1000C9F608952091E4059091C306213208F098
:101D20004AC08091C1058111FCCF32E03093C105DA
:101D300031E03093C0053FEF3093BF051092BE05F0
:101D40002093BD05A4ECB5E04DE955E0FA013E2F26
:101D5000341B321718F43D913193F9CF10929C0542
:101D600020919C05990F922B90939C0590919B0537
:101D7000913061F410929B0590919C059093BB006B
:101D80009091BC0093FDF8CF95EC01C095EE909337
:101D9000BC009091C1059230E1F39091BF059F3F47
:101DA00079F08091BF05803241F08091BF0580338A
:101DB00031F084E005C081E003C082E001C083E02F
:101DC0001092C3051092E4051092C2050895833065
:101DD00081F028F4813099F08230A1F008958730A5
:101DE000A9F08830B9F08430D1F4809180008F7DE3
:101DF00003C0809180008F7780938000089584B520
:101E00008F7702C084B58F7D84BD08958091B00026
:101E10008F7703C08091B0008F7D8093B0000895CC
:101E2000009769F0FC0101900020E9F73197AF01BC
:101E3000481B590BBC0185E996E00C94AD1A80E073
:101E400090E00895CF93C82F8091B1068F3F59F14C
:101E5000E091BB06F091BC0680819091C106982B61
:101E60009083E091BD06F091BE0620819091C2065C
:101E7000909592239083E091BB06F091BC0620815F
:101E80009091C1069095922390838C2F0E94540EBE
:101E9000E091BB06F091BC0690818091C106892B30
:101EA0008083CF9108958091AF0691E09093C20511
:101EB0008093C3061092C3051092E40560E082E8A7
:101EC00096E00E940D186C2F82E896E00E940D1893
:101ED000CF910C948A0EEF92FF920F931F93CF93A2
:101EE000DF9381E20E94220F80E00E94220F8FE7A1
:101EF0000E94220F82E20E94220F80E00E94220FA5
:101F000087E00E94220F8091B1068F3F79F1E09126
:101F1000BB06F091BC0690818091C106892B80831D
:101F2000E091BD06F091BE0690818091C206892B9A
:101F30008083E091BB06F091BC0690818091C10640
:101F4000809589238083CFE1D1E089910E94540E4E
:101F500085E0CF31D807C9F7E091BB06F091BC0608
:101F600090818091C106892B808330C0F090B800A9
:101F70008CE08093B800CFE1D1E0EE24E39480912F
:101F8000AF06E092C2058093C3061092C30510927B
:101F9000E40560E482E896E00E940D1800E010E09D
:101FA000FE01E00FF11F608182E896E00E940D18AB
:101FB0000F5F1F4F0031110599F70E948A0E60963E
:101FC00085E0CF31D807D9F6F092B800DF91CF91F4
:101FD0001F910F91FF90EF90089580E094E0EFE162
:101FE000F1E0DF019C011D9221503040E1F7E5E96D
:101FF000F6E0158614861786168681E0848B81E0CC
:1020000090E0938B828B918B808B08950C94100FB2
:10201000DF92EF92FF920F931F93CF93DF93EC0128
:10202000D62E00919F061091A00620919D0630911A
:102030009E06EE24E394F12C40E050E060E070E076
:1020400085E996E00E94660B20919D0630919E06E0
:102050000BE010E040E050E060E070E085E996E0E1
:102060000E94040B81E08093A9061092A8061092AA
:10207000A7061092A6061092A506DD20E1F0FE014B
:1020800001900020E9F73197EC1BFD0B26E02E9F15
:10209000C0012F9F900D112420919D0630919E0626
:1020A000281B390B369527953093A2062093A1065D
:1020B00082E090E006C082E090E09093A2068093D8
:1020C000A1069093A4068093A306CE010E94061059
:1020D00081E090E09093A8068093A7069093A606CF
:1020E0008093A506DF91CF911F910F91FF90EF9004
:1020F000DF9008958F929F92AF92BF920F931F939C
:10210000CF93DF93CDB7DEB7A1970FB6F894DEBFBC
:102110000FBECDBF19A2423008F44AE08E010F5D18
:102120001F4F842E912CA12CB12CA50194010E944B
:10213000B134E62FB901CA0101501109EA3014F493
:10214000E05D01C0E95CD801EC93232B242B252B07
:1021500061F7C8010E94100FA1960FB6F894DEBF78
:102160000FBECDBFDF91CF911F910F91BF90AF9068
:102170009F908F900895CF93C82F0E94ED0F8CE809
:1021800099E00E94CE1261E00E940810E5E9F6E0B5
:1021900085E0848B81E090E0938B828B918B808BA8
:1021A00084E190E095878487978786876C2F70E01D
:1021B00080E090E04AE00E947A100E946B0FCF917D
:1021C0000C94ED0FE0919506F09196060190F08148
:1021D000E02D682F85E996E00994CF92DF92EF9287
:1021E000FF920F931F93CF93DF93182FEB016A0198
:1021F0000E94ED0F8EE799E00E94CE1261E00E94EE
:10220000081081E090E09093A8068093A706909331
:10221000A6068093A50635E0E32EF12CF092A206E7
:10222000E092A1068CE090E09093A4068093A30630
:102230008FE699E00E94CE120E940610F092A2064C
:10224000E092A1064CE1E42EF12CF092A406E0927B
:10225000A30689E699E00E94CE120E94061086E24B
:1022600090E09093A2068093A106F092A406E092DB
:10227000A306612F67706F5F70E080E090E04AE036
:102280000E947A108DE9C8168FEFD806E9F08DE527
:1022900099E00E94CE120E9406100D2C000CEE0850
:1022A000FF08F7FE0CC08DE20E94E2106627772738
:1022B000CB016C197D098E099F094AE003C04AE0F1
:1022C000C701B6010E947A1085E090E09093A206C3
:1022D0008093A10604E210E01093A4060093A306E5
:1022E0008FE499E00E94CE120E94061086E290E0F0
:1022F0009093A2068093A1061093A4060093A306D0
:10230000BE0180E090E04AE00E947A1080919D0634
:1023100090919E068254910997FD01969595879517
:102320009093A2068093A10684E390E09093A40684
:102330008093A30683E499E00E94CE120E940610C7
:10234000DF91CF911F910F91FF90EF90DF90CF9091
:102350000C946B0FCF93DF93282F30E0F901E15DF0
:10236000F64F8491F901E55EF64FD491F901E95FEA
:10237000F64FC491CC2391F081110E94E70EEC2F0F
:10238000F0E0EE0FFF1FE350F74FA591B491EC91F1
:10239000ED2381E090E021F480E002C080E090E055
:1023A000DF91CF9108951F93CF93DF93282F30E0D3
:1023B000F901E15DF64F8491F901E55EF64FD491A4
:1023C000F901E95FF64FC491CC23C9F0162F8111B2
:1023D0000E94E70EEC2FF0E0EE0FFF1FED50F74FDD
:1023E000A591B4918FB7F894111105C09C91ED2F70
:1023F000E095E92302C0EC91ED2BEC938FBFDF91C8
:10240000CF911F910895CF93DF9390E0FC01E55E9B
:10241000F64F2491FC01E95FF64F8491882361F126
:1024200090E0880F991FFC01E751F74FC591D491B7
:10243000FC01ED50F74FA591B491611109C09FB710
:10244000F8948881209582238883EC912E230BC0F9
:10245000623061F49FB7F8943881822F809583238E
:102460008883EC912E2B2C939FBF06C08FB7F894D6
:10247000E8812E2B28838FBFDF91CF9108958E3076
:1024800008F08E508770806480937C0080917A0081
:10249000806480937A0080917A0086FDFCCF8091E1
:1024A00078002091790090E0922B08958F929F926E
:1024B000AF92BF92CF92DF92EF92FF926B017C01BD
:1024C0000E94D81A4B015C01C114D104E104F1044B
:1024D000F1F00E94D81ADC01CB0188199909AA09E8
:1024E000BB09883E9340A105B10570F321E0C21AF3
:1024F000D108E108F10888EE880E83E0981EA11C3F
:10250000B11CC114D104E104F10419F7DDCFFF902F
:10251000EF90DF90CF90BF90AF909F908F900895F5
:1025200061E08BE00C94D31160E08CE00E94D31149
:1025300060E08AE00E94D31161E08CE00E94D31138
:1025400060E08CE00C94D31160E08CE00E94D31129
:1025500061E08AE00E94D31161E08CE00E94D31117
:1025600060E08CE00C94D311E82FF0E0EF55F64FCB
:102570008491282F2F70205D90E044E095958795F9
:102580004A95E1F78A30910514F0895C01C0855BBA
:1025900090E0982F8827820F911D0895FC01A8ECE8
:1025A000B6E090E02491222331F09E3121F02D936A
:1025B00031969F5FF7CFE92FF0E0E853F94F208382
:1025C00088EC96E008950F931F93CF938C010E949F
:1025D000901260E08BE00E94D3110E9494120E943E
:1025E00094120E9494120E94A4120E949412C4E1B8
:1025F0000E949412C150E1F70E94901260E08BE0BB
:102600000E94D3110E94901260E08BE00E94D311CF
:102610000E94A4120E9494120E9494120E9494128A
:102620000E94A412C0E100FF03C00E94A41202C0D5
:102630000E94941216950795C150A9F70E94941212
:102640000E9494120E9494120E9494120E9490126E
:1026500060E08BE00E94D31160E08CE00E94D31117
:1026600060E08AE0CF911F910F910C94D311E0911B
:10267000780580910201E8130CC020917605309115
:1026800077058091E7069091E8062817390709F445
:1026900048C080917205E8131DC0209176053091E5
:1026A000770521153105B1F02F5D3140C9019695AF
:1026B000879556E0369527955A95E1F73695322F4E
:1026C0002227379527958F719927820F931F0E9494
:1026D000E31211C0F0E0EE0FFF1FE950FD4F8591AE
:1026E00094910E94E3128091780580937205109274
:1026F000770510927605809178058093020180918C
:102700007605909177059093E8068093E7060E94FE
:10271000FD1A6093C4067093C5068093C606909315
:10272000C70608950F931F93CF93DF93E091F505AC
:10273000F091F60582E08083E091F505F091F605D1
:102740001082E091F105F091F2051082E091F3051D
:10275000F091F40580E180831092FD05E091F90588
:10276000F091FA0586E08083E091F705F091F80595
:10277000808180618083E091F705F091F805808188
:1027800088608083E091F705F091F805808180688A
:102790008083E091F705F091F80580818F7D80833B
:1027A00061E08DE00E94031261E08DE00E94D31190
:1027B00061E086E00E94031261E086E00E94D3118E
:1027C00060E082E00E94031262E082E00E94D31186
:1027D00060E083E00E94031262E083E00E94D31174
:1027E00060E084E00E94031262E084E00E94D31162
:1027F00060E085E00E94031262E085E00E94D31150
:1028000061E08EE00E94031261E08FE00E940312FB
:1028100088B18C7F816088B981E08093060161E096
:102820008BE00E94031261E08AE00E94031261E0E3
:102830008CE00E94031282E190E00E94C819893165
:10284000974209F46BC0C0E0D0E06FEFCE010E9468
:10285000C4192196C11581E0D807B9F761E080E07D
:1028600090E00E94C41960E081E090E00E94C419E9
:1028700060E070E080E190E00E94DD196091090164
:102880008BE090E00E94C41960E08CE390E00E942D
:10289000C41960E08EE090E00E94C41960910801C4
:1028A0008CE090E00E94C4196AE570E082E090E05C
:1028B0000E94DD196CED70E084E090E00E94DD196B
:1028C0004AE050E06FE675E081E995E00E946234ED
:1028D00001E915E0C4E1D0E0F80161918F01CE017A
:1028E0000E94C4192196CE31D105B1F760917505CA
:1028F0008AE090E00E94C4196AE570E086E090E00A
:102900000E94DD196CED70E088E090E00E94DD1916
:1029100069E177E282E190E00E94DD1980E090E0D9
:102920000E94C61980931C0180931B0181E090E0F6
:102930000E94C61980937805803338F0109278058C
:1029400060E081E090E00E94C419809178050E94C7
:10295000440E80937905809178058093720580E11B
:1029600090E00E94C8199093770580937605885867
:102970009341883E934050F010927705109276056F
:1029800060E070E080E190E00E94DD190E94371362
:1029900000E410E0C0E0C8010E94C819803391052E
:1029A00030F09C0128583341283E334028F4CF5F53
:1029B0000E5F1F4FCA3079F7C0937305CC2359F0CF
:1029C0008CE390E00E94C6198C1718F4809374056C
:1029D00002C0109274058BE090E00E94C61991E04D
:1029E000811101C090E0909309018CE090E00E9479
:1029F000C61991E0811101C090E09093080101E9AE
:102A000015E0C4E1D0E0CE010E94C619F80181931F
:102A10008F012196CE31D105B1F782E090E00E947E
:102A2000C819909319018093180184E090E00E94E6
:102A3000C81990931701809316018AE090E00E94D4
:102A4000C6198093750586E090E00E94C81990939E
:102A500011018093100188E090E00E94C8199093C2
:102A60000F0180930E0181E080937A0592E09093AC
:102A7000B0069CE39093AF069091B1069F3F09F496
:102A8000BDC061E08091B3060E94031261E08091B5
:102A9000B5060E9403128091B506082E000C990B12
:102AA000FC01E95FF64FE491F0E0EE0FFF1FED50FF
:102AB000F74F259134913093BC062093BB06FC015F
:102AC000E55EF64FE491E093C1068091B306082ECF
:102AD000000C990BFC01E95FF64FE491F0E0EE0F7A
:102AE000FF1FED50F74F259134913093BE06209390
:102AF000BD06FC01E55EF64FE491E093C2068091CD
:102B0000B60681113EC061E08091B1060E940312B9
:102B100061E08091B2060E9403128091B206082EF5
:102B2000000C990BFC01E95FF64FE491F0E0EE0F29
:102B3000FF1FED50F74F259134913093BA06209343
:102B4000B906FC01E55EF64FE491E093C006809182
:102B5000B106082E000C990BFC01E95FF64FE491D9
:102B6000F0E0EE0FFF1FED50F74F259134913093B9
:102B7000B8062093B706FC01E55EF64FE491E093BA
:102B8000BF068091B606882309F45EC0CFB7F894DB
:102B90008091E606811127C0E1E1F9E08491E5E248
:102BA000F9E09491E82FF0E0EE0FFF1FE751F74FA7
:102BB000A591B491EC91E92321F461E08AE00E94AF
:102BC000D31161E08AE00E9403128CB580618CBD54
:102BD0008CB580648CBD61E08DE00E94031261E0E1
:102BE0008BE00E9403128091E6068F5F8093E606D9
:102BF000CFBF80E58CBD81E08DBD26C01092EA0676
:102C00001092E9061092C3051092E4051092C105D6
:102C10008093C00510929B0561E082E10E94D31170
:102C200061E083E10E94D3118091B9008E7F80938F
:102C3000B9008091B9008D7F8093B90088E48093BA
:102C4000B80085E48093BC008091B40687FD1EC067
:102C500061E00E94031261E08091B4060E94D311EA
:102C600061E070E080E090E00E94561260E08091A8
:102C7000B4060E94D3116AE070E080E090E00E9408
:102C8000561261E08091B4060E94D3118EEA0E9430
:102C9000220F85ED0E94220F80E80E94220F88EA11
:102CA0000E94220F8FE30E94220F83ED0E94220FC9
:102CB00080E00E94220F80E40E94220F8DE80E9493
:102CC000220F84E10E94220F80E20E94220F80E006
:102CD0000E94220F81EA0E94220F88EC0E94220F9C
:102CE0008AED0E94220F82E10E94220F81E80E9459
:102CF000220F8FEC0E94220F89ED0E94220F81EF9C
:102D00000E94220F8BED0E94220F80E40E94220F6E
:102D100084EA0E94220F86EA0E94220F8EE20E941D
:102D2000220F8FEA0E94220F0E946B0F60ED77E066
:102D300080E090E00E9456120E94ED0F85E10E9413
:102D40003F12059714F41092750560E08DE00E9423
:102D5000D31180911C01843011F483E003C08A30C8
:102D600019F484E080931D01DF91CF911F910F91A1
:102D70000895FC01918D828D981761F0828DDF019D
:102D8000A80FB11D5D968C91928D9F5F9F73928F5E
:102D900090E008958FEF9FEF0895FC01918D828D53
:102DA000981731F0828DE80FF11D858D90E0089520
:102DB0008FEF9FEF0895FC01918D228D892F90E078
:102DC000805C9F4F821B91098F739927089585EE30
:102DD00095E00E94DB1621E0892B09F420E0822F88
:102DE0000895FC01848DDF01A80FB11DA35ABF4FC8
:102DF0002C91848D90E001968F739927848FA689FA
:102E0000B7892C93A089B1898C9180648C93938D20
:102E1000848D981306C00288F389E02D80818F7D10
:102E200080830895EF92FF920F931F93CF93DF93C8
:102E3000EC0181E0888F9B8D8C8D981305C0E8890B
:102E4000F989808185FD24C0F62E0B8D10E00F5F7F
:102E50001F4F0F731127E02E8C8DE8120CC00FB698
:102E600007FCFACFE889F989808185FFF5CFCE018B
:102E70000E94F116F1CF8B8DFE01E80FF11DE35A90
:102E8000FF4FF0820B8FEA89FB898081806207C047
:102E9000EE89FF896083E889F98980818064808375
:102EA00081E090E0DF91CF911F910F91FF90EF9023
:102EB0000895CF93DF93EC01888D8823C9F0EA89C8
:102EC000FB89808185FD05C0A889B9898C9186FD23
:102ED0000FC00FB607FCF5CF808185FFF2CFA88920
:102EE000B9898C9185FFEDCFCE010E94F116E7CF15
:102EF000DF91CF91089580E090E0892B29F00E9426
:102F0000E71681110C9400000895089581E090E087
:102F10003091EA062091E906321710F480E090E043
:102F200091958195910908958091EA069091E9061D
:102F3000891730F48F5F8093EA0680E090E008956F
:102F40008FEF9FEF08958091E90690E02091EA06C7
:102F5000821B9109089585ED8093BC008091BC008F
:102F600084FDFCCF1092C105089540910F07262FD4
:102F700030E0240F311D21323105DCF42091C105F0
:102F80002430C9F4FC0180E090E0861758F43091B9
:102F90000F072191DC01A351B94FA30FB11D2C9351
:102FA0000196F3CF80910F07680F60930F0780E0C1
:102FB000089581E0089582E00895CF92DF92EF9224
:102FC000FF920F931F93CF93DF937C01262F972FB0
:102FD0008A018091C205882391F0C62FD72F6E01F8
:102FE000C40ED51ECC15DD0571F06991D701ED91A8
:102FF000FC910190F081E02DC7010995F3CF642F7A
:10300000822F0E94B517C801DF91CF911F910F91B8
:10301000FF90EF90DF90CF900895CF93DF931F92B2
:10302000CDB7DEB769832091C2052223D1F020916C
:10303000E405203240F021E030E0FC0133832283BC
:1030400080E090E015C08091C305E82FF0E0EC53DC
:10305000FA4F998190838F5F8093C3058093E40535
:1030600005C061E0CE0101960E94B51781E090E0B5
:103070000F90DF91CF9108950E945D341F920F92BF
:103080000FB60F9211242F933F934F935F936F933B
:103090007F938F939F93AF93BF93EF93FF9385EEAF
:1030A00095E00E94F116FF91EF91BF91AF919F9132
:1030B0008F917F916F915F914F913F912F910F90E1
:1030C0000FBE0F901F9018951F920F920FB60F9280
:1030D00011242F938F939F93EF93FF93E091F50526
:1030E000F091F6058081E091FB05F091FC0582FDF1
:1030F00012C090818091FE058F5F8F732091FF0534
:10310000821751F0E091FE05F0E0EB51FA4F958FF8
:103110008093FE0501C08081FF91EF919F918F9177
:103120002F910F900FBE0F901F9018951F920F9226
:103130000FB60F9211242F933F934F935F936F938A
:103140007F938F939F93AF93BF93EF93FF93809160
:10315000B900887F803609F49CC068F5883209F48C
:103160005BC090F4803109F454C038F4882309F42A
:10317000F6C0883009F44DC0F6C0883109F44CC05F
:10318000803209F45DC0EFC0803409F468C048F4AF
:10319000803309F455C0883309F0E5C08093BF053A
:1031A000D8C0803509F44FC0883509F45DC0883433
:1031B00009F0D9C0D6C0883909F4C7C0A8F4883747
:1031C00009F467C038F4883609F463C0803709F41D
:1031D00060C0C9C0883809F4B8C0803909F45FC03C
:1031E000803809F0C0C05BC0803B09F486C038F469
:1031F000803A09F466C0883A09F47FC0B4C0803CC4
:1032000009F4A7C0883C09F4A4C0883B09F48AC02B
:10321000AAC080919C0510C09091BE058091BD050B
:10322000981770F5E091BE0581E08E0F8093BE0582
:10323000F0E0E356FA4F80818093BB0085EC86C0B6
:103240008093BF058EC0E091BE0581E08E0F809314
:10325000BE058091BB00F0E0E356FA4F8083909169
:10326000BE058091BD056EC0E091BE0581E08E0F68
:103270008093BE058091BB00F0E0E356FA4F808357
:103280008091C00581116DC081E080939B0584EA27
:1032900061C083E08093C10510923307CFCF809146
:1032A0003307803208F051C0E091330781E08E0F80
:1032B000809333078091BB00F0E0ED5EF84F808390
:1032C000BDCF85EC8093BC001092C105809133077F
:1032D000803230F4E0913307F0E0ED5EF84F108279
:1032E0006091330770E0E0911107F091120783E1DC
:1032F00097E009951092330736C084E08093C105AA
:103300001092100710920F07E0910D07F0910E0731
:10331000099580910F07811105C081E080930F0707
:103320001092ED06E091100781E08E0F8093100758
:10333000F0E0E351F94F80818093BB00909110073A
:1033400080910F07981708F479CF85E88093BC0027
:103350000AC085EC8093BC001092C10504C0109295
:10336000BF050E94AB17FF91EF91BF91AF919F9165
:103370008F917F916F915F914F913F912F910F901E
:103380000FBE0F901F9018950C9479340C947134E3
:103390001F93CF93DF93EC010E94C619182FCE0123
:1033A00001960E94C619282F30E0922F8827810F9E
:1033B000911DDF91CF911F9108950F931F93CF938C
:1033C000DF931F92CDB7DEB78C0179830E94C419B9
:1033D0007981672FC80101960F90DF91CF911F91DE
:1033E0000F910C94C41985EE95E00E94DB16181617
:1033F000190684F485EE95E00E94B9168D3511F416
:1034000082E003C08B3521F481E080937B05089531
:1034100010927B0580E00895CF92DF92EF92FF92A9
:103420000F931F93CF93DF936C010091730510E00E
:1034300080E4E82EF12CC0E0D0E0C017D1075CF4A6
:10344000C7010E94C81922E0E20EF11C8C159D05EF
:1034500029F02196F2CF8FEF9FEF01C0CE01DF91CF
:10346000CF911F910F91FF90EF90DF90CF90089533
:1034700090917305891780F490E08096880F991FCA
:103480000E94C8198033910548F09C0128583341A7
:10349000283E334008F408958FEF9FEF0895CF93AF
:1034A000DF93EC0161E08DE00E94D311809109016E
:1034B000882321F060E086E00E94D311BE0176955A
:1034C000679580E090E00E94561260E08DE00E94D7
:1034D000D31161E086E0DF91CF910C94D31160911C
:1034E000780580912205681731F06093220581E00C
:1034F00090E00E94C41960917605709177058091E3
:103500002005909121056817790741F070932105F6
:103510006093200580E190E00C94DD19089580917E
:103520007605909177050097B9F4E0917805809140
:103530001F05E81769F0E0931F05F0E0EE0FFF1F8D
:10354000E35CFD4F859194919093EC068093EB069C
:103550008091EB069091EC060895CF92DF92EF9266
:10356000FF920F931F93CF93DF936C017A018B012E
:10357000C0E0D0E0CE15DF0589F0D8016D918D0156
:10358000D601ED91FC910190F081E02DC6010995E5
:10359000892B11F47E0102C02196ECCFC701DF9187
:1035A000CF911F910F91FF90EF90DF90CF900895F2
:1035B0003FB7F8948091390790913A07A0913B0763
:1035C000B0913C0726B5A89B05C02F3F19F0019686
:1035D000A11DB11D3FBFBA2FA92F982F8827820F99
:1035E000911DA11DB11DBC01CD0142E0660F771FE9
:1035F000881F991F4A95D1F708952FB7F8946091C5
:1036000035077091360780913707909138072FBFA3
:1036100008951F920F920FB60F9211242F933F938C
:103620008F939F93AF93BF93809135079091360707
:10363000A0913707B09138073091340723E0230F6A
:103640002D3720F40196A11DB11D05C026E8230FDA
:103650000296A11DB11D20933407809335079093E6
:103660003607A0933707B0933807809139079091B8
:103670003A07A0913B07B0913C070196A11DB11DEF
:103680008093390790933A07A0933B07B0933C0788
:10369000BF91AF919F918F913F912F910F900FBE4E
:1036A0000F901F901895CF93DF93CDB7DEB72B9770
:1036B0000FB6F894DEBF0FBECDBF789484B582609C
:1036C00084BD84B5816084BD85B5826085BD85B5C6
:1036D000816085BD80916E00816080936E00109244
:1036E00081008091810082608093810080918100BF
:1036F0008160809381008091800081608093800050
:103700008091B10084608093B1008091B0008160AD
:103710008093B00080917A00846080937A008091D9
:103720007A00826080937A0080917A008160809331
:103730007A0080917A00806880937A001092C100AC
:103740000E949213B5E02B2E312C83E00E94AA1127
:10375000892B09F054C010928705109288051092A9
:10376000890510928A0582E390E00E944F1A64E670
:1037700070E080E090E00E94561282E390E00E94A8
:103780004F1A64E670E080E090E00E945612C12C6F
:1037900083E00E94AA11892B59F42AE0C21641F055
:1037A00064E670E080E090E00E945612C394F0CF8F
:1037B00020911D01298380911C01811103C081E0AA
:1037C00080931C011092860532E33A8310E071E287
:1037D000872E912CEBE26E2E712CF5E34F2E512C9F
:1037E000ABE0AA2ED0901D0149E04C1510F00C94CE
:1037F000F12C86E080931C018FEF80931A011092C8
:103800007F0585E00E94AA11892B19F486E0809338
:103810001C0180917A0510911C01811105C08091D5
:103820001A01181709F4C6C310927A05812F90E087
:10383000FC013197EA30F10508F0B8C3EC5CFF4FAA
:103840000C941E3282E080931B0110927905EFE503
:10385000F3E0859194918093780581E080938305CE
:103860000E94ED0F10928F06109292061092910610
:1038700010929406109293061230A1F481E591E023
:103880000E94CE1261E00E9408103092A20620929F
:10389000A1068CE090E09093A4068093A3068BE4AD
:1038A00091E013C080E491E00E94CE1261E00E949A
:1038B00008103092A2062092A1068CE090E090932E
:1038C000A4068093A30682E391E00E94CE120E9498
:1038D000061020919D0630919E06EE24E394F12C73
:1038E00004E110E044E150E060E070E085E996E03A
:1038F0000E94B50B40919F065091A0064B50510974
:1039000020919D0630919E068A0160E070E085E975
:1039100096E00E94B50B80919F069091A0060997B2
:1039200022E030E03093A2062093A1069093A406F3
:103930008093A3068DE291E00E94CE120E940610B1
:1039400080919F069091A006099727E330E030937D
:10395000A2062093A1069093A4068093A30688E272
:1039600091E00E94CE120E94061080919F069091D5
:10397000A006099720919D0630919E062951310994
:103980003093A2062093A1069093A4068093A306E9
:1039900083E291E00E94CE120E9406100E946B0FFB
:1039A00005C3133079F50E94FD1A60938705709363
:1039B00088058093890590938A0580911B01833047
:1039C00029F063E080E090E00E94C41980911B011F
:1039D0009FEF980F923020F090911A01983059F48F
:1039E00081E090E00E94C619809378050E94440E01
:1039F0008093790502C0843069F4109277051092A3
:103A0000760508C0109287051092880510928905E6
:103A100010928A0510911C018FEF809390060E94EE
:103A2000ED0F1A3019F48EE891E009C0133019F443
:103A300082E891E004C0113039F483E791E00E94FC
:103A4000CE1261E00E94081081E090E09093A806F9
:103A50008093A7069093A6068093A50620919D06C5
:103A600030919E0601E010E044E150E060E070E03B
:103A700085E996E00E946E0620919D0630919E0693
:103A800040E250E060E070E085E996E00E946E065A
:103A90003092A2062092A1068CE090E09093A406BA
:103AA0008093A306EE24E394F12C04E110E021E6D8
:103AB00030E04BE050E061E670E085E996E00E947E
:103AC000B50B8DE691E00E94CE120E94061011E324
:103AD00008E0E02EF12CF092A206E092A10627E188
:103AE00030E03093A4062093A306812F0E94E210B9
:103AF0003FE0E30EF11C1F5F193369F720919D062B
:103B000030919E06EE24E394F12C04E210E044E2AE
:103B100050E060E070E085E996E00E94B50B4091CE
:103B20009F065091A0064B50510920919D0630915F
:103B30009E068A0160E070E085E996E00E94B50B80
:103B400080919F069091A006099722E030E0309383
:103B5000A2062093A1069093A4068093A30688E66C
:103B600091E00E94CE120E94061080919F069091D3
:103B7000A006099727E330E03093A2062093A10620
:103B80009093A4068093A30683E691E00E94CE1250
:103B90000E94061080919F069091A006099720919F
:103BA0009D0630919E06295131093093A20620933B
:103BB000A1069093A4068093A3068EE591E00E944F
:103BC000CE120E9406100E946B0F81E080937D054B
:103BD000E9C16091780581E090E00E94C41960918C
:103BE00009018BE090E00E94C419609108018CE00B
:103BF00090E00E94C419A1E9EA2EA5E0FA2E04E1A2
:103C000010E0F70161917F01C8010E94C4190F5FA4
:103C10001F4F0E311105A9F7609175058AE090E0FC
:103C20000E94C41980911A01853009F466C0809100
:103C30001B018A3009F46AC000917605109177055E
:103C40000115110519F40091780510E0C8010E94D2
:103C50000C1A97FD11C080937405682F8CE390E0D7
:103C60000E94C419809174058F5F0E94BB1060E2AE
:103C700073E080E090E054C1F0E4EF2EF12CC12C11
:103C8000D12CC7010E94C8198033910558F088587B
:103C90009341883E934030F0809173058F5F80930D
:103CA000730513C02FEFC21AD20A32E0E30EF11CE3
:103CB0004AE0C416D10429F780917405CC24C3943A
:103CC000C80E89E08C1508F4C12C8C2D90E08096EC
:103CD000B801880F991F0E94DD19C09274056C2DE0
:103CE0008CE390E00E94C4190091740510E00F5F0E
:103CF0001F4F0E948F1AA80104C00E948F1A4DE91D
:103D00005FEFBC01809178050E94ED1080911B014E
:103D10008A3009F0F4C080911A018F3F09F0EFC09A
:103D2000D090740580917305D81608F0E8C00E9401
:103D30008F1A5C010E94ED0F85EC91E00E94CE127B
:103D400061E00E94081081E090E09093A8068093C3
:103D5000A7069093A6068093A5063092A20620920D
:103D6000A1065CE0E52EF12CF092A406E092A306F9
:103D700087EB91E00E94CE120E94061005E510E04C
:103D80001093A2060093A106F092A406E092A30667
:103D9000B50180E090E04AE00E947A103092A206DD
:103DA0002092A10664E1E62EF12CF092A406E092A6
:103DB000A3068AEA91E00E94CE120E940610109398
:103DC000A2060093A106F092A406E092A30661E089
:103DD0006D0D70E080E090E04AE00E947A108091E2
:103DE0009D0690919E068254910997FD01969595A6
:103DF00087959093A2068093A10684E390E0909328
:103E0000A4068093A3068CE991E00E94CE120E9442
:103E100006100E946B0F64EF71E080E090E00E945A
:103E200056129090740599E0991508F44BC0E92C4E
:103E3000F12C3701E0E26E0E711C660C771C8701D5
:103E400068018FEFC81AD80A9AE0C916D104B9F0F0
:103E50005301F2E0AF0EB11CC5010E94C8198033B6
:103E6000910530F09C0128583341283E334048F4F6
:103E7000BC01C3010E94DD1935018601E1CF09E0D3
:103E800010E0C80180966FEF7FEF880F991F0E94A6
:103E9000DD1900937305E016F106A1F491100AC034
:103EA000109273051092740560E08CE390E00E941C
:103EB000C41925C06FEF690D609374058CE390E021
:103EC0000E94C419809174050E94381A97FD12C08F
:103ED0008F3F910519F014F00C94692F80937805A9
:103EE00010927705109276050E94440E8093790512
:103EF0000E946F1A809174058F5F0E94BB1015E0BD
:103F000084E690E00E944F1A64E670E080E090E062
:103F10000E9456121150A1F76CE271E080E090E02F
:103F20000E94561280911B0180931C0181E08093B6
:103F30007A053CC00E94FD1A60938705709388053E
:103F40008093890590938A058AE02EC00E94FD1A0D
:103F500060938705709388058093890590938A05FF
:103F600080911B01843011F164E080E090E00E94B8
:103F7000C41980911B018150823020F080911A0178
:103F8000883081F481E090E00E94C6198093780522
:103F90008093720580E190E00E94C81990937705A4
:103FA0008093760580911C0180931B0180911C01F8
:103FB00080931A01809107018823D1F010920701A4
:103FC00082E390E00E944F1A62E370E080E090E0AC
:103FD0000E94561282E390E00E944F1A62E370E062
:103FE00080E090E00E94561282E390E00E944F1A17
:103FF00080911C01982F9D7F993069F0843059F091
:1040000080911C01873009F01AC580907505B1E2D6
:10401000AB2EB12C57C30E948F1A7C01809178057A
:10402000E82FF0E0EE0FFF1FE35CFD4F2591349188
:104030002E153F0521F40E94B4124C0102C0812CC0
:10404000912CD09075050E94ED0F84E08093A90615
:1040500001E010E01093A8060093A7061093A606AF
:104060000093A50682E0A82EB12CB092A206A092E1
:10407000A1061092A4061092A306B70180E090E07A
:104080004AE00E947A1081E08093A9061092A2066D
:104090001092A1068CE190E09093A4068093A30671
:1040A00081E995E00E94061082E08093A90682E6ED
:1040B00090E09093A2068093A106B092A406A092ED
:1040C000A3061093A8060093A7061093A6060093D4
:1040D000A5068114910431F0892D0E94E210882DEB
:1040E0000E94E21081E08093A906E12CF12C0BE103
:1040F00010E022E330E04BE150E060E070E085E961
:1041000096E00E94B50B85E10E943F12059754F19D
:1041100082E690E09093A2068093A10684E190E06D
:104120009093A4068093A30681E090E09093A60666
:104130008093A5061092A8061092A706E1E0DE166D
:1041400059F0DE1630F0F2E0DF120CC08EED91E097
:1041500005C08AEE91E002C084EE91E00E94CE128A
:104160000E9406101092A6061092A506CC24C394B5
:10417000D12CD092A806C092A70640919F065091DC
:10418000A0064B515109EE24E394F12C0DE010E010
:1041900027E030E060E070E085E996E00E94040BE3
:1041A00080919F069091A0064897D092A206C09257
:1041B000A1069093A4068093A3068CED91E00E9443
:1041C000CE120E9406106AE085E996E00E940F0A6E
:1041D0001092A6061092A506D092A806C092A70635
:1041E00040919F065091A0064D50510927E030E0C4
:1041F00060E070E085E996E00E94040B80919F06E4
:104200009091A0060B97D092A206C092A10690931F
:10421000A4068093A3068AED91E00E94CE120E942C
:1042200006100E946B0F0E94FD1A60938705709321
:1042300088058093890590938A05AA24A394B12CBC
:10424000B7E78B2E912C0E94ED0DC82E809185052D
:104250008823B9F0409087055090880560908905C3
:1042600070908A0528EE420E23E0521E611C711CDC
:104270000E94FD1A461657066806790610F40C943B
:104280006F2F409087055090880560908905709049
:104290008A05411451046104710479F00E94FD1AE9
:1042A00030E7430E37E1531E611C711C461657065A
:1042B0006806790610F40C94752F82E00E945F0C5A
:1042C000D82E81E00E945F0C898370900601809156
:1042D0001C018B3009F068C00E94ED0F4981442E0B
:1042E000512C612C712CA3019201215031094109FB
:1042F0005109A4E7B0E00E94A63423E630E040E094
:1043000050E00E948734DA01C9010396A11DB11D56
:10431000282F30E0EE24E394F12C0EE110E04EE182
:1043200050E060E070E085E996E00E94040B27E72A
:1043300030E04EE150E060E070E085E996E00E94F8
:10434000660B84E08093A906B092A806A092A70607
:10435000B092A606A092A506E4E1F0E0F093A206D2
:10436000E093A1061092A4061092A3064AE0C301AE
:10437000B2010E947A108FEF91E00E94CE120E944B
:1043800006101092A2061092A1061092A406109296
:10439000A306F981F23310F068E101C069E185E913
:1043A00096E00E940F0A61C185E10E943F120091D0
:1043B0009F061091A00605970CF4B9C02981822FA1
:1043C00090E0A0E0B0E09C01AD012150310941092D
:1043D0005109A4E7B0E00E94A63423E630E040E0B3
:1043E00050E00E948734DA01C9010396A11DB11D76
:1043F000482E512C940124193509A8014B5151091B
:10440000B201695F7F4FE12CF12C0DE010E085E9EE
:1044100096E00E94040B40919F065091A00631E067
:104420004B51510973120BC0EE24E394F12C92010D
:1044300067E070E085E996E00E94040B1CC0E12C67
:10444000F12C0DE010E027E730E067E070E085E94F
:1044500096E00E94040B40919F065091A0064B519C
:104460005109EE24E394F12C920167E070E085E9B4
:1044700096E00E94660B8D2D90E0A0E0B0E09C01DC
:10448000AD012150310941095109A4E7B0E00E9472
:10449000A63423E630E040E050E00E948734DA01A1
:1044A000C9010396A11DB11D482E512C9401241958
:1044B000350940919F065091A0064D505109B20117
:1044C000695F7F4FE12CF12C0DE010E085E996E06B
:1044D0000E94040B40919F065091A00682E04D502F
:1044E0005109781207C0EE24E394F12C920167E0A1
:1044F00070E082C0E12CF12C0DE010E027E730E005
:1045000067E070E085E996E00E94040B40919F0609
:104510005091A0064D505109EE24E394F12C9201E4
:1045200067E070E085E996E00E94660B69C0109232
:10453000A8061092A7061092A6061092A506A8013A
:104540004B515109EE24E394F12C03E110E029E1F1
:1045500030E060E070E085E996E00E94040B809115
:104560009F069091A0060D97B092A206A092A10678
:104570009093A4068093A3068AEF91E00E94CE1246
:104580000E9406108C2D90E0A0E0B0E09C01AD01EF
:104590002150310941095109A4E6B0E00E94A63436
:1045A00023E630E040E050E00E948734DA01C901A0
:1045B0000196A11DB11D682E712C25E630E026194B
:1045C000370940919F065091A00643515109B3010C
:1045D000675E7F4FE12CF12C85E996E00E94040B89
:1045E00040919F065091A0064B515109EE24E3944F
:1045F000F12C930169E170E085E996E00E94040BDB
:1046000093E19C1578F10E94FD1A2AEF30E040E01A
:1046100050E00E94B13421E030E06D377105810532
:10462000910510F020E030E03093A6062093A50617
:104630001092A8061092A70680919F069091A0065E
:104640004297EDE2F0E0F093A206E093A10690938A
:10465000A4068093A3068FEE91E00E94CE120E94E2
:10466000061003C085E10E943F120E946B0F82E09A
:104670000E94AA11892B99F010917B05113079F0D5
:1046800084E00E94AA11892B51F0123041F010925F
:104690007C0583E00E94AA11019709F4D4CD809192
:1046A0001B0180931C0191E090938405843011F0EC
:1046B0000C94ED2C83E00E94AA11892B11F40C9428
:1046C000ED2C9ECC809275050E94ED0F83E292E066
:1046D0000E94CE1261E00E94081020919D06309148
:1046E0009E06FAE08F9EA0011124445F5F4FEE24E6
:1046F000E394F12C0AE010E060E070E085E996E0D8
:104700000E94040B81E090E0811002C080E090E004
:104710009093A8068093A7069093A6068093A5067B
:104720003092A2062092A1062DE030E03093A4063C
:104730002093A3068EE192E00E94CE120E94061002
:1047400081E090E031E0831202C080E090E090933D
:10475000A8068093A7069093A6068093A50630929C
:10476000A2062092A10687E190E09093A406809390
:10477000A30683E192E00E94CE120E94061081E01F
:1047800090E0E2E08E1202C080E090E09093A806F4
:104790008093A7069093A6068093A5063092A20662
:1047A0002092A106B092A406A092A30688E092E00F
:1047B0000E94CE120E94061081E090E09093A8061D
:1047C0008093A7069093A6068093A50620919D0648
:1047D00030919E0640919F065091A0064551510987
:1047E000EE24E394F12C0BE010E060E070E085E94A
:1047F00096E00E94660B80919F069091A0064397D9
:104800003092A2062092A1069093A4068093A3065C
:1048100085E092E00E94CE120E94061080919F06D1
:104820009091A00609973092A2062092A10690933B
:10483000A4068093A30683E092E00E94CE120E9419
:1048400006100E946B0F0E94ED0D82E00E945F0C2B
:10485000982E81E00E945F0C7090060190E0A0E02D
:10486000B0E09C01AD012150310941095109ABE68D
:10487000B0E00E94A63423E630E040E050E00E9421
:104880008734DA01C9010196A11DB11DC82ED12CB2
:104890002CE630E02C193D0940919F065091A0066E
:1048A00043515109B6016E5E7F4FE12CF12C07E0B8
:1048B00010E085E996E00E94040B40919F0650911C
:1048C000A006F1E0435151097F120BC0EE24E3949E
:1048D000F12C960162E170E085E996E00E94040BFC
:1048E0001BC0E12CF12C07E010E0960162E170E0C2
:1048F00085E996E00E94040B40919F065091A00626
:1049000043515109EE24E394F12C960162E170E0E9
:1049100085E996E00E94660B892D90E0A0E0B0E06A
:104920009C01AD012150310941095109ABE6B0E0CC
:104930000E94A63423E630E040E050E00E94873435
:10494000DA01C9010196A11DB11DC82ED12C2CE69A
:1049500030E02C193D0940919F065091A006495026
:104960005109B6016E5E7F4FE12CF12C07E010E09B
:1049700085E996E00E94040B40919F065091A006A5
:1049800022E04950510972120BC0EE24E394F12C3D
:10499000960162E170E085E996E00E94040B1BC07D
:1049A000E12CF12C07E010E0960162E170E085E96E
:1049B00096E00E94040B40919F065091A00649503A
:1049C0005109EE24E394F12C960162E170E085E94F
:1049D00096E00E94660B0E946B0F83E00E94AA1172
:1049E000019779F482E00E94AA11019751F484E0C2
:1049F0000E94AA11019729F40E94F319882309F44F
:104A000022CF83E00E94AA11892B11F00C947F2FF2
:104A100010E032E0381514F00C94892F812C82E3D9
:104A200090E00E944F1A68EC70E080E090E00E94F5
:104A30005612111147CE80911B0180931C01809169
:104A40001C018A3009F0BEC000917305002309F4EF
:104A500070C080918605882341F10E94F00D0E946C
:104A6000ED0D0E94FD1A6093870570938805809371
:104A7000890590938A0582E00E94AA1111E0892B92
:104A800029F080917B05813009F010E084E00E94DC
:104A9000AA11892B11F40C94A62F80917B058230EA
:104AA00011F00C949F2F0C94A62F6AE080E090E008
:104AB0000E94C41981E080938605809176059091CB
:104AC0007705009721F40091780510E001C08C0172
:104AD000C8010E940C1A97FD03C08093740505C09D
:104AE000809174050E94381A8C0117FD16C00F3F83
:104AF000110509F064F4009378051092770510927F
:104B00007605802F0E94440E8093790504C010938F
:104B10007705009376050E946F1A809174058F5F68
:104B20000E94BB1064EF71E080E090E00E9456129A
:104B300049C00E94ED0F83E392E00E94CE1261E033
:104B40000E94081083E08093A90681E090E0909392
:104B5000A8068093A7069093A6068093A50684E1F5
:104B600090E09093A2068093A1069093A406809370
:104B7000A3068DE292E00E94CE120E9406100E94CF
:104B80006B0F68EE73E080E090E00E94561289E0BF
:104B900080931C018091760590917705892B11F007
:104BA00064E001C063E060931B0180E090E00E943C
:104BB000C41980911B01833011F083E001C082E0B1
:104BC00080931D0140911C014A87443069F5809112
:104BD000760590917705892B69F4E0917805F0E0EE
:104BE000EE0FFF1FE35CFD4F859194919093770545
:104BF0008093760582E00E94AA1111E0892B29F0AA
:104C000080917B05813009F010E084E00E94AA11B8
:104C1000892B11F40C94A92F80917B05823011F01F
:104C20000C943F300C94A92F1A851D7F113009F088
:104C300067C38091760590917705892B41F010929A
:104C40007705109276050E943713109385050E9410
:104C5000F00D0E94ED0DD82E0E94F319F82E8093CE
:104C60007B0500917805802F0E94440EE82E182FB6
:104C7000809379052A85233009F073C082E00E9471
:104C8000AA11892B19F031E0F31228C00E94FD1AF5
:104C900060938705709388058093890590938A05B2
:104CA00082E390E00E944F1A68EC70E080E090E0B0
:104CB0000E94561210927B050F5F0093780581E0E9
:104CC0008E0D803314F40C94443010927905003327
:104CD00010F01092780581E08093850584E00E94B1
:104CE000AA11892B21F080917B05823051F50E9419
:104CF000FD1A6093870570938805809389059093CA
:104D00008A0582E390E00E944F1A68EC70E080E030
:104D100090E00E94561210927B0590917805915078
:104D20009093780580917905815087FD8FE280937B
:104D30007905903318F08FE28093780581E08093B5
:104D40008505809108018111B0C0E09179050E2E92
:104D5000000CFF0BE15AFC4F8591949180937805EC
:104D6000A4C04A85413009F0A0C08091810581111D
:104D700069C080918205811144C08CE38D1508F0D3
:104D800040C0809180058D3308F03BC04093810581
:104D9000EE24E39480910301882321F01F5F1033F8
:104DA00024F021C0115017FD1EC0E12F012E000C70
:104DB000FF0BE15AFC4FA590B490A09278050E9499
:104DC00037130E94F00D0E94ED0DD81628F00093C5
:104DD00078050E94371307C010937905E0927D058E
:104DE0000A2DD82ED7CF0E94FD1A609387057093A5
:104DF00088058093890590938A0581E080938505D5
:104E000021C01092820580910301882339F081E04E
:104E10008E0D803354F01092790509C0EA94E7FCB6
:104E200003C0E092790503C08FE280937905E09199
:104E300079050E2E000CFF0BE15AFC4F85919491E1
:104E40008093780582E00E94AA1111E0892B11F06D
:104E5000F11210E084E00E94AA11892B11F40C9445
:104E6000483092E0F91611F40C9448301123D9F02F
:104E70001093030182E390E00E944F1A10927B0589
:104E800068EC70E080E090E00E94561281E0809330
:104E90008205109281051092870510928805109264
:104EA000890510928A05D0928005809087059090A0
:104EB0008805A0908905B0908A0581149104A10409
:104EC000B10409F10E94FD1A9501840108571C4E96
:104ED0002F4F3F4F061717072807390728F4E2E33B
:104EE000ED1510F40C944D300E94FD1AF0E78F0E72
:104EF000F7E19F1EA11CB11C86169706A806B906ED
:104F000010F40C944D3010917805809102018113BA
:104F100005C080917D05882309F4EFC1909081053B
:104F20000E948F1A2C01C090790580901C018091FD
:104F30009006C81609F4A3C08C1510F483E001C0D4
:104F40008FEF8093000181E090E09093A60680931C
:104F5000A5061092A8061092A70684E290E090930E
:104F6000A2068093A1068CE090E09093A406809323
:104F7000A306183218F08DEE92E016C0103218F029
:104F800083EE92E011C0183118F089ED92E00CC068
:104F9000103118F08FEC92E007C0183018F085EC53
:104FA00092E002C08BEB92E00E94CE120E940610AB
:104FB000177084E0682E712CA12CB12C212F30E0C9
:104FC0003B832A83EE24E394F12C8A819B81A816EB
:104FD000B90611F0E12CF12C0BE010E02EE030E0EE
:104FE00045E150E0B30185E996E00E94040B81E0C1
:104FF00090E0EA81FB81AE16BF0611F480E090E0FC
:105000009093A8068093A7069093A6068093A50682
:10501000C30104969093A2068093A10627E130E095
:105020003093A4062093A30681E38A0D0E94E21028
:105030003FEFA31AB30A4FE0640E711C88E0A81674
:10504000B10409F0BFCF85E690E09093A20680936B
:10505000A1068CE090E09093A4068093A30681E0E3
:1050600090E09093A6068093A5061092A806109251
:10507000A706B20180E090E04AE00E947A10009119
:105080009D0610919E06035011094D2C512C612C48
:10509000712C91E0491A510861087108C801012E6C
:1050A000000CAA0BBB0BBC01CD0161507109810939
:1050B0009109A30192010E94E63123E630E040E02D
:1050C00050E00E948734DA01C9010196A11DB11D8B
:1050D000A82EB12C98012A193B09B5016F5F7F4FAB
:1050E000E12CF12C03E010E041E250E085E996E08C
:1050F0000E94040BEE24E394F12C950141E250E070
:1051000061E070E085E996E00E94040BADE0B0E05C
:10511000A30192010E94A63423E630E040E050E073
:105120000E94873429013A01EFEF4E1A5E0A6E0A97
:105130007E0AF3E0CF9E5001112424E0A20EB11CA0
:105140000EE010E00419150940919F065091A00649
:105150004A515109E12CF12C22E030E0B50185E9FA
:1051600096E00E94040B40919F065091A0064C507F
:10517000510944195509EE24E394F12C820122E0EF
:1051800030E0B50185E996E00E94040B31E083121E
:10519000A0C040919F065091A0064A51510985E058
:1051A000C89EB0011124759567956C5F7F4F809103
:1051B0000001680F711D87FD7A95E12CF12C0EE03E
:1051C00010E021E030E085E996E00E94040B409178
:1051D0009F065091A0064A51510922E030E061E05B
:1051E00070E085E996E00E94040B40919F06509183
:1051F000A00644515109EE24E394F12C8A0122E0E7
:1052000030E061E070E085E996E00E94B50B4091E6
:105210009F065091A0064A51510960919D067091D8
:105220009E0663507109E12CF12C0EE010E022E0A3
:1052300030E085E996E00E94040B40919F06509172
:10524000A0064451510920919D0630919E06B90156
:1052500063507109EE24E394F12C8A0185E996E00C
:105260000E94B50B80919D0690919E061092A60615
:105270001092A50621E030E03093A8062093A706FF
:1052800084559109992089F097FD01969595879508
:105290009093A2068093A10682E090E09093A406EA
:1052A0008093A3068CEA92E010C097FD0196959535
:1052B00087959093A2068093A10682E090E0909358
:1052C000A4068093A3068DE992E00E94CE120E946C
:1052D0000610C09290060E946B0F10927D0580917F
:1052E0008105882351F00E94FD1A60938705709311
:1052F00088058093890590938A0510928405F5C1ED
:105300009A85923019F0983009F0EFC180918305A9
:105310008823A1F0109283051092770510927605EC
:1053200010917805E12FF0E0EE0FFF1FE950FD4FDF
:10533000859194910E94E312109302010E94F00D56
:105340000E94ED0D8983809178050E94B4129B83A1
:105350008A830E948F1A9D838C83E0911201F091C1
:105360001301FF83EE8320911401309115013987D9
:105370002887309179053B8780909F069090A00602
:1053800080919006381709F4CDC04981842F90E0B0
:10539000A0E0B0E09C01AD01215031094109510963
:1053A000ADE1B0E00E94A63423E630E040E050E0FA
:1053B0000E94873429013A018FEF481A580A680A77
:1053C000780AEB8595E0E99F60011124D594C79494
:1053D0005601F4E0AF0EB11C0EE110E004191509FE
:1053E000A4014A525109E12CF12C22E030E0B50130
:1053F00085E996E00E94040BA4014C505109441920
:105400005509EE24E394F12C820122E030E0B5014D
:1054100085E996E00E94040B40919F065091A006FA
:105420004A525109B601695F7F4FE12CF12C0EE120
:1054300010E021E030E085E996E00E94040B2A8527
:10544000283009F472C0809190063B85381708F027
:1054500040C010928F06809191069091920600971D
:10546000C1F121E030E03093A6062093A50610920A
:10547000A8061092A70624E230E03093A2062093FB
:10548000A1060CE010E01093A4060093A306892F58
:105490000E94E210809191060E94E21084E390E065
:1054A0009093A2068093A1061093A4060093A306EE
:1054B000609193067091940680E090E04AE00E942B
:1054C0007A10109292061092910610929406109201
:1054D000930649814D3308F476C080918F06841776
:1054E00078F440938F068A819B81909392068093F3
:1054F0009106EC81FD81F0939406E093930663C0DE
:105500008091010190E0099620919D0630919E06C0
:105510002C503109821793070CF455C08CE380930B
:10552000010151C02A852830A1F6BEE1CB2ED12C35
:10553000D092A206C092A1060CE010E01093A4063F
:105540000093A306EE24E394F12CF092A606E092D9
:10555000A5061092A8061092A7068BE593E00E947C
:10556000CE120E940610D092A206C092A1061093FD
:10557000A4060093A30628853985B90180E090E050
:105580004AE00E947A1085E590E09093A20680930D
:10559000A1061093A4060093A306F092A606E0923B
:1055A000A5061092A8061092A70687E593E00E9430
:1055B000CE120E940610EE81FF81BF0180E090E0D4
:1055C0004AE00E947A100E946B0FFB85F0939006D0
:1055D000809179058F3224F48F5F809379056CC0B8
:1055E0001092790580911C01883009F065C0809186
:1055F0007E059FEF980F90937E0581115DC06091AD
:10560000140170911501709319016093180182E0E3
:1056100090E00E94DD1920911201309113018091D8
:10562000140190911501F901E81BF90B63E070E09A
:105630000E94F631E617F70748F0309317012093E0
:105640001601B90184E090E00E94DD1985E10E9415
:105650003F1205973CF160910C0170910D01709320
:1056600011016093100186E090E00E94DD19209105
:105670000A0130910B0180910C0190910D01F9010B
:10568000E81BF90B63E070E00E94F631E617F707BC
:1056900048F030930F0120930E01B90188E090E0AB
:1056A0000E94DD1980E090E00E94C61980931C01E1
:1056B00088EE93E00E944F1A0E94F319182F8093EE
:1056C0007B0582E00E94AA11892B09F4EBC41130FA
:1056D00009F4E8C4E09179050E2E000CFF0BE15AA5
:1056E000FC4F859194918093780580911C018530C1
:1056F00009F071C1CC24CA94DC2C1982E1E28E2E0F
:10570000912CFBE2AF2EB12CA5E36A2E712CCA823C
:1057100040900801509009010E94ED0F8EED93E03A
:105720000E94CE1261E00E94081020919D063091E7
:105730009E0689819AE08902A0011124445F5F4F8F
:10574000EE24E394F12C0AE010E060E070E085E9DB
:1057500096E00E94040B81E090E0E981E11102C033
:1057600080E090E09093A8068093A7069093A60609
:105770008093A5063092A2062092A1062DE030E08B
:105780003093A4062093A30686ED93E00E94CE12E8
:105790000E940610442019F08CEC93E002C082ECC9
:1057A00093E00E94CE120E94061081E090E03981C1
:1057B000313011F480E090E09093A8068093A70622
:1057C0009093A6068093A5063092A2062092A10689
:1057D00087E190E09093A4068093A3068AEB93E080
:1057E0000E94CE120E940610552019F086EB93E01D
:1057F00002C082EB93E00E94CE120E94061081E06C
:1058000090E0E981E23011F480E090E09093A80606
:105810008093A7069093A6068093A5063092A206D1
:105820002092A1069092A4068092A3068AEA93E0B1
:105830000E94CE120E940610FA81F7FD48C0209106
:105840009D0630919E062A523109E12CF12C08E088
:1058500010E041E250E069E270E085E996E00E94E4
:10586000040B2A81422E022E000C550836E023023A
:10587000B0011124625D7F4FEE24E394F12C27E008
:1058800030E041E250E085E996E00E94040B01E936
:1058900015E0E12CF12C81E090E0E414F50411F422
:1058A00080E090E09093A8068093A7069093A606C8
:1058B0008093A506F80181918F010E94E210FFEF0D
:1058C000EF1AFF0A2AE0E216F10429F704C081E981
:1058D00095E00E94061081E090E03981333011F4A8
:1058E00080E090E09093A8068093A7069093A60688
:1058F0008093A5063092A2062092A106B092A4063B
:10590000A092A3068BE993E00E94CE120E9406109B
:1059100081E090E04981443011F480E090E0909380
:10592000A8068093A7069093A6068093A5063092BA
:10593000A2062092A1067092A4066092A3068FE8A8
:1059400093E00E94CE120E9406100E946B0F12E399
:10595000115009F4C8C483E00E94AA110197A9F468
:1059600082E00E94AA11019781F484E00E94AA11AA
:10597000019759F40E94F319811107C064E670E0A1
:1059800080E090E00E945612E3CF83E00E94AA11CB
:10599000892B09F04CC48981823009F42BC40CF0A6
:1059A0001FC4811113C49091080181E0892780935D
:1059B000080111E082E390E00E944F1A66E970E06E
:1059C00080E090E00E945612FFEFCF16DF0609F448
:1059D00049C411119CCE0E9437130E947B170C946E
:1059E000A51B80918505882321F0109285050E94D2
:1059F0006F1A111110C080911C01833061F48091E5
:105A00008405811108C089E080931C0181E08093A6
:105A100084050C94FC1BE9818E2FEE0F990BAA0BC9
:105A2000BB0B8830910590F5FC01E25CFF4F0C94B4
:105A30001E3281E080931C0112C0F2E0F0931C0141
:105A400081E080938305B3C023E020931C0107C04D
:105A500034E030931C0103C04AE040931C01D9801C
:105A6000A6C085E080931C0115C085E10E943F120D
:105A7000059724F097E090931C010CC0A0921C01A4
:105A8000E7E0E98307C0A0921C0104C0F981F5306A
:105A90000CF48DC02BEFB22E2981B20E0E94ED0FB7
:105AA00086EB90E00E94CE1260E00E9408102091E8
:105AB0009D0630919E068AE0B89EA0011124445FA5
:105AC0005F4FEE24E394F12C0AE010E060E070E018
:105AD00085E996E00E94040B81E090E0B11002C0DD
:105AE00080E090E09093A8068093A7069093A60686
:105AF0008093A5063092A2062092A106EDE0F0E088
:105B0000F093A406E093A3068BEA90E00E94CE12E5
:105B10000E94061081EA90E00E94CE120E940610B8
:105B200068E185E996E00E940F0A85E10E943F1234
:105B30000597FCF081E090E0F1E0BF1202C080E048
:105B400090E09093A8068093A7069093A606809372
:105B5000A5063092A2062092A10627E130E03093FC
:105B6000A4062093A30687E990E00E94CE120E942B
:105B7000061081E090E032E0B31202C080E090E0D5
:105B80009093A8068093A7069093A6068093A506F7
:105B90003092A2062092A1069092A4068092A306BB
:105BA0008CE890E00E94CE120E940610BFC00E94B6
:105BB000ED0F8EE091E00E94CE1260E00E9408108E
:105BC00020919D0630919E0699818AE0989FA001C0
:105BD0001124445F5F4FEE24E394F12C0AE010E0BF
:105BE00060E070E085E996E00E94040B81E090E0BF
:105BF000E981E11102C080E090E09093A8068093D3
:105C0000A7069093A6068093A5063092A20620923E
:105C1000A1062DE030E03093A4062093A30684E093
:105C200091E00E94CE120E94061081E090E039813E
:105C3000313011F480E090E09093A8068093A7069D
:105C40009093A6068093A5063092A2062092A10604
:105C500087E190E09093A4068093A30687EF90E0FD
:105C60000E94CE120E94061081E090E0E981E230AD
:105C700011F480E090E09093A8068093A70690939B
:105C8000A6068093A5063092A2062092A1069092C5
:105C9000A4068092A3068BEE90E00E94CE120E9492
:105CA000061081E090E0F981F33011F480E090E09B
:105CB0009093A8068093A7069093A6068093A506C6
:105CC0003092A2062092A1067092A4066092A306CA
:105CD0008FED90E00E94CE120E94061081E090E0CD
:105CE0002981243011F480E090E09093A8068093FD
:105CF000A7069093A6068093A5063092A20620924E
:105D0000A1065092A4064092A30685ED90E00E9461
:105D1000CE120E9406108BEC90E00E94CE120E94E0
:105D2000061069E185E996E00E940F0A0E946B0F58
:105D300083E00E94AA11892B19F432E33A83F8CF49
:105D400082E00E94AA11892BC1F384E00E94AA116B
:105D5000892B99F30E94F319813079F30E94F3198A
:105D6000823059F34A8141504A834423F9F083E059
:105D70000E94AA110197A9F482E00E94AA1101973A
:105D800081F484E00E94AA11019759F40E94F3194A
:105D9000811107C064E670E080E090E00E94561236
:105DA000E1CF83E00E94AA11892BF1F549814830A7
:105DB00009F45FC083E00E94AA11892B71F08091E1
:105DC0001B01823039F480911D01833011F484E08D
:105DD00001C083E080931C0111C0D0921D0180910D
:105DE0001C01813059F480938205809181058823BC
:105DF00019F01092810502C01092800584E690E0AF
:105E00000E944F1A62E370E080E090E00E94561218
:105E100084E690E00E944F1A62E370E080E090E038
:105E20000E9456120C94FC1B82E00E94AA11892B3E
:105E300009F4B7C110917B05113009F4B2C184E0B7
:105E40000E94AA11892B09F4BDC1123009F4BAC10C
:105E5000998198300CF4A0C1198282E390E00E94ED
:105E60004F1A68EC70E080E090E00E945612F2E376
:105E7000FA8311E00C94F21B62E370E07093190155
:105E8000609318014CE251E05093170140931601C2
:105E90002CED30E030931501209314018AE590E059
:105EA000909313018093120170931101609310017C
:105EB00050930F0140930E0130930D0120930C017C
:105EC00090930B0180930A0183E080937E050C94EC
:105ED000251C90937705809376050C94781F10927B
:105EE00085050E946F1A0C9441211092870510922B
:105EF00088051092890510928A050C945D2182E034
:105F00000E94AA11892BA9F010917B05113049F448
:105F100010C087FC02C00C940F2522E0822E0C9446
:105F20000F2584E00E94AA11892B39F0123011F458
:105F300004C08A9411E00C9409258394FBCF1111BD
:105F4000C6C089E080931C010C94E2251111F9CFA1
:105F5000C8C0111196C00E94FD1A60938705709306
:105F600088058093890590938A0580917C0581112D
:105F70000EC082E390E00E944F1A88EC90E090936C
:105F800005018093040181E080937C0511C080911C
:105F90000401909105018531910514F0449704C0E6
:105FA000181619062CF401979093050180930401AB
:105FB000E0900401F09005011E141F043CF4B701A9
:105FC0000F2C000C880B990B0E94561210927B0527
:105FD00080917605909177051123F1F01E141F042E
:105FE00014F401960BC00A966AE070E00E94F63144
:105FF0002AE0269FC001279F900D112490937705DA
:10600000809376058091760590917705803797414A
:1060100010F18FE697E11BC001971E141F0454F086
:106020006AE070E00E94F6312AE0269FC001279FB7
:10603000900D1124909377058093760580917605D5
:10604000909177058838934130F488E893E19093F4
:10605000770580937605612F80917605909177057D
:106060000E94100E182F809378050E94440E809392
:1060700079051093720581E08093850536CB111167
:106080006ACF10927C0531CB809379050C946726FA
:1060900011110C9453270C94382789E080931C012C
:1060A0000C94832782E390E00E944F1A68EC70E022
:1060B00080E090E00E9456128FEF80931A011092B8
:1060C000790581E08093830510927B0503CB023034
:1060D000B8F08091740561E0680F601758F060E0D7
:1060E00009C0023068F080917405882309F451C01A
:1060F0006FEF680F609374058CE390E00E94C41901
:106100000E94FD1A60938705709388058093890526
:1061100090938A05809174050E94381A97FD23C0D8
:106120008F3F910509F05CF4809378051092770514
:10613000109276050E94440E8093790510C09093CA
:10614000770580937605612F0E94100E182F80939B
:1061500078050E94440E80937905109372050E9481
:1061600037130E946F1A809174058F5F0E94BB10D5
:1061700068EC70E080E090E00E94561282E390E0CC
:106180000E944F1A68EC70E080E090E00E94561286
:10619000D8CE6FEF600FAECF97FF5FCEE7E0E98319
:1061A0005CCE1981812F8150898385E10E943F1245
:1061B00005970CF04DCE8981863009F049CE1250FA
:1061C000198346CE99819F5F998342CE813009F031
:1061D0003EC080910901E9818E2780930901E9CBB6
:1061E0009981933099F0943091F586E080931C0169
:1061F00010E0E0CBFFEFCF1ADF0A2AE0C216D1048D
:106200000CF4D7CBCC24CA94DC2CD3CB1AE089E194
:1062100090E00E944F1A69E170E080E090E00E94F7
:1062200056121150A1F788E080931C01C3CB82E085
:106230000E94AA11892B21F010917B05113079F56C
:10624000EFEFCE16DE0699F5398131503983998109
:1062500011E095302CF497FFADCBE4E0E983AACBB5
:106260001982A8CB83E00E94AA11892B09F4A6CB3E
:1062700082E00E94AA11892B09F4A0CB84E00E943D
:10628000AA11892B09F49ACB0E94F319813009F4E1
:1062900095CB0E94F319823009F490CB9ACB84E01D
:1062A0000E94AA11892BB9F0123089F614C0F601A8
:1062B000EF56FA4F80818F5F8E375CF040E240836B
:1062C000C6CFF601EF56FA4F8081815080320CF430
:1062D0008DE78083BCCFFFEFCF16DF0691F7898172
:1062E0008F5F8983B4CF80911B0180931C0173CB96
:1062F000E5EEF5E01382128288EE93E0A0E0B0E0D4
:1063000084839583A683B7832BE335E03183208391
:1063100025EC30E03587248724EC30E0378726876A
:1063200020EC30E0318B208B21EC30E0338B228B62
:1063300022EC30E0358B248B26EC30E0378B268B3B
:10634000118E128E138E148EE2E8F6E01382128202
:1063500084839583A683B7838BE495E091838083C0
:10636000EEE8F6E08FEF82831082118214821382AE
:1063700016821582E5E9F6E01382128240E850E0C9
:106380005583448320E430E0378326835187408758
:1063900033872287158A158614861786168691E01C
:1063A000948B2FEF3FEF338B228B318B208B968B8F
:1063B000178A118E108E2BE535E031832083848F70
:1063C00080A3868F858F84E0878F0895DB018F936C
:1063D0009F930E94A634BF91AF91A29F800D911D03
:1063E000A39F900DB29F900D11240895AA1BBB1B73
:1063F00051E107C0AA1FBB1FA617B70710F0A61BC5
:10640000B70B881F991F5A95A9F780959095BC01E5
:10641000CD01089597FB072E16F4009407D077FD61
:1064200009D00E94F63107FC05D03EF49095819585
:106430009F4F0895709561957F4F0895EE0FFF1F50
:106440000590F491E02D09945058BB27AA270E948B
:106450003C320C948D330E947F3338F00E94863397
:1064600020F039F49F3F19F426F40C947C330EF499
:10647000E095E7FB0C947633E92F0E949E3358F3A6
:10648000BA17620773078407950720F079F4A6F519
:106490000C94C0330EF4E0950B2EBA2FA02D0B01F7
:1064A000B90190010C01CA01A0011124FF27591B59
:1064B00099F0593F50F4503E68F11A16F040A22F5F
:1064C000232F342F4427585FF3CF469537952795D0
:1064D000A795F0405395C9F77EF41F16BA0B620BCF
:1064E000730B840BBAF09150A1F0FF0FBB1F661F16
:1064F000771F881FC2F70EC0BA0F621F731F841F59
:1065000048F4879577956795B795F7959E3F08F07E
:10651000B0CF9395880F08F09927EE0F9795879540
:1065200008950E94A5320C948D330E94863358F052
:106530000E947F3340F029F45F3F29F00C947633BA
:1065400051110C94C1330C947C330E949E3368F338
:106550009923B1F3552391F3951B550BBB27AA271C
:1065600062177307840738F09F5F5F4F220F331F56
:10657000441FAA1FA9F335D00E2E3AF0E0E832D01E
:1065800091505040E695001CCAF72BD0FE2F29D021
:10659000660F771F881FBB1F261737074807AB07F3
:1065A000B0E809F0BB0B802DBF01FF2793585F4F68
:1065B0003AF09E3F510578F00C9476330C94C13339
:1065C0005F3FE4F3983ED4F3869577956795B7954A
:1065D000F7959F5FC9F7880F911D9695879597F955
:1065E0000895E1E0660F771F881FBB1F62177307CE
:1065F0008407BA0720F0621B730B840BBA0BEE1FE3
:1066000088F7E09508950E940A336894B1110C94BC
:10661000C13308950E94A63388F09F5798F0B92F90
:106620009927B751B0F0E1F0660F771F881F991FC7
:106630001AF0BA95C9F714C0B13091F00E94C03376
:10664000B1E008950C94C033672F782F8827B85F86
:1066500039F0B93FCCF3869577956795B395D9F71F
:106660003EF490958095709561957F4F8F4F9F4F29
:106670000895E89409C097FB3EF490958095709535
:1066800061957F4F8F4F9F4F9923A9F0F92F96E97E
:10669000BB279395F695879577956795B795F111F3
:1066A000F8CFFAF4BB0F11F460FF1BC06F5F7F4F90
:1066B0008F4F9F4F16C0882311F096E911C07723A2
:1066C00021F09EE8872F762F05C0662371F096E8AB
:1066D000862F70E060E02AF09A95660F771F881F7A
:1066E000DAF7880F9695879597F9089597F99F6738
:1066F00080E870E060E008959FEF80EC089500244A
:106700000A941616170618060906089500240A9416
:1067100012161306140605060895092E0394000C9C
:1067200011F4882352F0BB0F40F4BF2B11F460FF2B
:1067300004C06F5F7F4F8F4F9F4F089557FD905854
:10674000440F551F59F05F3F71F04795880F97FB35
:10675000991F61F09F3F79F08795089512161306EF
:106760001406551FF2CF4695F1DF08C0161617061E
:106770001806991FF1CF8695710561050894089553
:10678000E894BB2766277727CB0197F908950E94E5
:10679000393408F48FEF08950E94DF330C948D3361
:1067A0000E947F3338F00E94863320F0952311F049
:1067B0000C9476330C947C3311240C94C1330E94D6
:1067C0009E3370F3959FC1F3950F50E0551F629F64
:1067D000F001729FBB27F00DB11D639FAA27F00D3A
:1067E000B11DAA1F649F6627B00DA11D661F829F61
:1067F0002227B00DA11D621F739FB00DA11D621F46
:10680000839FA00D611D221F749F3327A00D611D62
:10681000231F849F600D211D822F762F6A2F112444
:106820009F5750409AF0F1F088234AF0EE0FFF1F77
:10683000BB1F661F771F881F91505040A9F79E3FCE
:10684000510580F00C9476330C94C1335F3FE4F330
:10685000983ED4F3869577956795B795F795E79524
:106860009F5FC1F7FE2B880F911D9695879597F92D
:106870000895990F0008550FAA0BE0E8FEEF1616D1
:106880001706E807F907C0F012161306E407F50724
:1068900098F0621B730B840B950B39F40A2661F098
:1068A000232B242B252B21F408950A2609F4A1403B
:1068B000A6958FEF811D811D089581E090E0F894E9
:1068C0000C94E234FB01DC014150504048F001904F
:1068D0000D920020C9F701C01D9241505040E0F7D1
:1068E0000895F999FECF92BD81BDF89A992780B598
:1068F0000895262FF999FECF1FBA92BD81BD20BD04
:106900000FB6F894FA9AF99A0FBE01960895052EDB
:1069100097FB1EF400940E949E3457FD07D00E94FE
:10692000B13407FC03D04EF40C949E34509540953E
:10693000309521953F4F4F4F5F4F0895909580952B
:10694000709561957F4F8F4F9F4F08950E94D3346C
:10695000A59F900DB49F900DA49F800D911D1124B3
:106960000895A1E21A2EAA1BBB1BFD010DC0AA1F90
:10697000BB1FEE1FFF1FA217B307E407F50720F0A8
:10698000A21BB30BE40BF50B661F771F881F991F23
:106990001A9469F760957095809590959B01AC016C
:1069A000BD01CF010895A29FB001B39FC001A39F75
:1069B000700D811D1124911DB29F700D811D112438
:0869C000911D0895F894FFCF2A
:1069C800033CFF01C80001010101DC005A00DC00A2
:1069D8005A00DC005A00DC005A0002010102FF00E4
:1069E800000000000000000000000000000000009F
:1069F800000000000000008080C0E0E0E0D0A0F8C7
:106A080050A878C0B850E814F880788078807880EA
:106A1800708060804080008000000000000000005E
:106A2800000000000000000000000000000000005E
:106A3800000000000000000000000000000000004E
:106A4800000000000000000000000000000000003E
:106A5800000000000000000000000000000000002E
:106A6800000000000000000000000000000080C0DE
:106A7800E0F0F8FCFEFFFFFFFFFFFFFFFFFFFFFE58
:106A8800FDFFF5EBDEB57BCE790E094FC84FA8CBDD
:106A9800B46B8CEB0A0B0ACAAA6A946890608000EF
:106AA80000000000000000000000000000000000DE
:106AB80000000000000000000000000000000000CE
:106AC80000000000000000000000000000000000BE
:106AD80000000000000000000000000000000000AE
:106AE8000000000000000000000000E0F8FEFFFFCA
:106AF800FFFFFFFFFFFFFFFFFFFFFFFFFFFFFFFF9E
:106B0800FFFFFFFFFFFFFFFFF5E0E0E4E6E4E6AD8F
:106B1800F65DAAFFA0E060AF54FBA45FA857FA4552
:106B2800BC50C00000000000000000000000000091
:106B3800000000000000000000000000000000004D
:106B4800000000000000000000000000000000003D
:106B5800000000000000000000000000000000002D
:106B6800000000000000000000E0FFFFFFFFFFFF43
:106B7800FFFFFFFFFFFFFFFFFFFFFFFFFFFFFFFF1D
:106B8800FFFFFFFFFFFFFFFFFFFFFFFFFFFFFFFF0D
:106B9800FFFFFFFEFFFEFDFFFDFFFAF5FFF5FEF527
:106BA800FFF5FEF5000000000000000000000000F6
:106BB80000000000000000000000000000000000CD
:106BC80000000000000000000000000000000000BD
:106BD80000000000000000000000000000000000AD
:106BE80000000000000000000017FFFFFFFFFFFF8C
:106BF800FFFFFFFFFFFFFFFFFFFFFFFFFFFFFFFF9D
:106C0800FFFFFFFFFFFFFFFFFFFFFFFFFFFFFFFF8C
:106C1800FFFFFFFFFFFFFFFFFFFFFFFFFFFFFFFF7C
:106C2800FFFFFF7F010000000000000000000000DF
:106C3800000000000000000000000000000000004C
:106C4800000000000000000000000000000000003C
:106C5800000000000000000000000000000000002C
:106C68000000000000000000000001073F7FFFFF58
:106C7800FFFFFFFFFFFFFFFFFFFFFFFFFFFFFFFF1C
:106C8800FFFFFFFFFFFFFFFFFFFFFFFFFFFFFFFF0C
:106C9800FFFFFFFFFFFFFFFFFFFFFFFFFFFFFFFFFC
:106CA8007F1F070000F0F8A8B8F000FCFE9800FE6F
:106CB800FE08F8F800F0F8A8B8F000FEFE00FAFAAE
:106CC80000008000F0F888989800F0F88898F8603C
:106CD800D0F81818F8F808F8F000000000000000D4
:106CE8000000000000000000000000000000010398
:106CF800071F3F7F7FFFFFFFFFFFFFFFFFFFFFFF34
:106D0800FFFFFFFFFFFFFFFFFFFFFFFFFFFFFFFF8B
:106D1800FFFFFFFFFFFFFFFFFF7F3F3F0F0703015D
:106D28000000000000000101010000000101000155
:106D38000000000100000101010000000100000145
:106D48000001010000010101000000010101000033
:106D58000001000001000001010000000000000027
:106D6800000000000000000000000000000000001B
:106D78000000000000000101030707070F0F1F1F95
:106D88001F1F1F3F3F3F3F3F3F3F1F3F1F1F1F0F1B
:106D98000F0F0707030301010000000000000000B7
:106DA80000000000000000000000000000000000DB
:106DB80000000000000000000000000000000000CB
:106DC80000000000000000000000000000000000BB
:106DD800000000000000000000000000000000FFAC
:106DE800FFFFFF01000000000103070F1F3F7F00A6
:106DF80080C0E0F0F8FCFE000000001217AD1ADBBE
:106E080016B916CD165917000000000D18DD17A386
:106E180017941786178517000000000F0AAD1ACAC5
:106E280007B50B14056E06660B040BE60A68085FC7
:026E3800000058
:00000001FF
